:10000000F01F0010415500003F5500003F55000013
:100010003F5500003F5500003F5500000000000024
:100020000000000000000000000000003F5500003C
:100030003F550000000000003F5500004D24000027
:1000400055220000552200005522000055220000D4
:1000500055220000552200005522000055220000C4
:1000600055220000552200005522000055220000B4
:10007000552200003D5500003D550000C100000024
:10008000152500002D2500004127000059270000FC
:100090003D5500009D2800003D5500003D550000E5
:1000A0003D5500003D5500003D5500003D55000008
:1000B0003D5500003D5500003D5500003D550000F8
:1000C000554B10B51A6801321A60544B1A68544BDC
:1000D000D2B2302A69D01ADC182A44D012DC082A9D
:1000E00032D0102A00D094E04E4A002111604E49CF
:1000F0000A68501C08604D49895C4D4AC9B21160BC
:10010000282287E0202A63D0282A32D081E0482A9A
:100110005ED004DC382A51D0402A53D079E0502AEE
:1001200060D0582A75D13F490A68501C0860404980
:1001300008684049C0B288543F4A0221FF3111602B
:1001400080221021D20563E0374A00211160116836
:10015000481C1060354A515C354AC9B211602822EA
:100160001A6001223CE030490A68501C08602F499F
:1001700009E02D4A314910680968884207D21168A0
:10018000481C1060294A515C294AC9B240E02C4AF7
:1001900011688022D205002901D0202138E02649AB
:1001A0000220FF300860102132E08022D2051021A9
:1001B000116008221A608122520011E08221490058
:1001C0001D4A25E01E4A1168042201291AD11DE0AA
:1001D0008022D2051021116008221A600422FF3209
:1001E000154B17E00F4A1168481C1060104804684E
:1001F0001048E4B244541068114A116804220139CD
:10020000884203D28021C9050A6002E01A6000E03A
:10021000116008221A6010BD900200100400004016
:1002200018000040840200108C020010B40400107A
:1002300008000040A404001088020010C40400104C
:10024000A00400101B4B02211A6810B50A431A6063
:10025000194B20211A68041C0A431A60174B1849CD
:100260001A680A401A601868012210431860154B7A
:1002700018680140196019680A431A60124B6C2211
:100280001A60124B1249186805F0E0F9114A106023
:10029000114A1060022C02D1104BA0221A60104BA0
:1002A000802212021A6080234022DB0501201A609E
:1002B00010BDC046048004408080044030400440AB
:1002C000F8FCFFFF34400440180000409804001080
:1002D000400D030014000040100000400C000040DE
:1002E00000E100E0034B1B689A06FBD5024B186047
:1002F0007047C0461480004000800040FFFFFFFFB1
:100300007FB5051C00200C1C01F07EFA002801D0EE
:1003100002F09AFE00262660281C2E60211C01F0A7
:10032000A1FA301C01F070FAB04207D002F08CFE46
:100330002660281C2E60211C01F094FA0C4B1B78BF
:10034000002B13D00B4B2A6818680B49824203D14B
:1003500020680D68A84209D01A60236801A80B60C4
:10036000064902F0CDFC01A802F072FD7FBDC04637
:10037000880300103C010010400100107457000079
:1003800038B5051C0C1C281C211C02F05BF8024B24
:100390001B68002BF7D138BD6802001008B502F0C9
:1003A00085F808BD08B500230B60036001F05AFA18
:1003B00008BD000010B502F00FFE0D4B00201968BB
:1003C00002F034FA002002F021FA002002F0FEF9D7
:1003D000084B01241C60084B201C198802F0E2F82D
:1003E000201C02F0CFF8201C02F0ACF810BDC04673
:1003F00094040010800200109C04001037B50C24F7
:100400000120032102F01EF8684601A9FFF778FFDA
:10041000009D002D02D1013C002CF1D1FFF7CAFF55
:10042000281C3EBD08B5002002F0E0F9012002F0D2
:1004300099F802F0D7FD08BD38B5051C0C1CFFF774
:10044000B9FF064AF823DB000121D150281C211CEA
:1004500004F044FAFFF7E6FF38BDC046D4040010AC
:1004600010B5041CFFF7A6FF201C04F06FF9041C54
:10047000FFF7D8FF201C10BD08B50020FFF7F0FFE4
:1004800008BD000008B5021C0249034802F02CFC1C
:1004900008BDC0468A5700008257000037B501F0FA
:1004A00029F80322164B1748002101F011F901F039
:1004B0002BF8FFF7E1FF1448FFF7E4FF134B144A52
:1004C00000241A601D1C2B689C4211DA02F0C8FA45
:1004D000002803D001F096FD00240FE00A2001F06F
:1004E000E5FF684601A9FFF70BFF009B002B05D035
:1004F000FFF7C2FF074802F0F7FB37BD0134E2E720
:100500002861000093570000A257000084030010E8
:1005100070170000A85700001B4B73B5041C1B4943
:10052000186805F093F81A4900901A4A1A4B201CD3
:1005300002F0E6FB01F072FA002812D001F08AFA0C
:10054000FA218900061C05F081F8051C201C02F028
:1005500028FC124B20186B431149F3182A1C02F097
:10056000CFFB201C02F01DFC0E4B20181B68002B3B
:1005700002D003DA0C4A02E00C4A00E00C4A0D49B2
:1005800002F0BEFB73BDC0469804001040420F004D
:10059000B95700008A570000C657000018FCFFFF3B
:1005A000CA57000050010010B6570000B3570000B2
:1005B000D8610000D557000070B5051C0E1C141C36
:1005C00000F098FF301C291C0022064B01F080F837
:1005D000201C01210922044B01F07AF800F094FF5D
:1005E00070BDC046286100002061000007B51449B5
:1005F000144A0120FFF7E0FF642001F057FF72B6B4
:10060000114B00211960114B01221A6019601A6008
:10061000196801221142FBD00D4B68461A600D4B40
:100620008022196852020A431A600B4B80211A6813
:100630000A431A603923009301A9084B984707BD64
:10064000DD570000D86100007080044074800440D1
:10065000788004408080044038820440F11FFF1FEE
:1006600000B5084B89B01A78074B68461B780749D4
:1006700002F046FB01206946054AFFF79DFF09B0DD
:1006800000BDC04644010010010000100D580000DC
:100690001B580000F0B52A4C2A4D237885B00193F1
:1006A0002F78FFF7DDFFFFF7E7FE002602A803A97A
:1006B000FFF726FE029800282BD0C0B201F022F8E6
:1006C00040280CD004D830280ED0392817D01BE091
:1006D000462830D049280DD0412815D126E02B7866
:1006E0003E2B11D8013303E02B78002B0CD0013BBB
:1006F0002B7009E02378062B06D8013303E023781A
:10070000002B01D0013B237000F0E0FEFFF7A8FFB3
:100710000026029B002B02D0C82001F0C7FE042057
:1007200003210136FFF72CFE1D2EBFDD019B2F702C
:10073000237000F0CBFEFFF79FFE05B0F0BDC04672
:10074000010000104401001038B5051C0C1C00F01D
:100750009CFE291C221C0120FFF72EFF054B064A98
:10076000002199501A1C94321168F522D200995038
:1007700038BDC046D4040010A407000010B590B0E6
:100780006846FFF7C9FE00F0B5FE084C0121684637
:100790000A1C231C00F09CFF054801210922231C90
:1007A00000F096FF00F0B0FE10B010BD2061000018
:1007B0002F58000000B52D228DB0002800D02B222C
:1007C00068460D4902F09CFA04A802F0CFFC012013
:1007D000694604AAFFF7F0FE03200021FFF7D0FDD1
:1007E0000220FFF73DFE0028EED00A200021FFF78F
:1007F000C7FD0DB000BDC04668580000F8B5041C28
:10080000161C0D1C002702F0B1FC211C1431E774EA
:10081000681C02F0CFFA00F06DFE201C04213A1C87
:100820000A4B00F055FF0A4C281C04210922231C06
:1008300000F04EFFBE4205D0064878210922231C55
:1008400000F046FF00F060FEF8BDC04628610000E1
:10085000206100001162000010B58CB0FFF70CFEA3
:10086000124902A802F0A6FA04A802A90022FFF782
:10087000C5FF2E24FF34002204A802A9FFF7BEFF03
:100880000020032101F0DEFD0023684601A9019349
:100890000093FFF735FD009B002B02D1013C002C9B
:1008A000E9D1FFF7E9FD0CB010BDC04670A1000012
:1008B000F0B5002493B00594FFF7DEFD02229623E5
:1008C00001940392271C5B00029300F013FE019B2E
:1008D0009A4E002B6DD10AAD281C02F047FC019AFC
:1008E000EA742A746A73AA72EA712A71002C01D11F
:1008F000012F05D1281C04210022331C00F0E8FE42
:100900008F4D331C281C1E21002200F0E1FE8B4E6F
:10091000012C01D1012F06D168462D30252100225E
:10092000331C00F0D5FE281C33210022331C00F0BC
:10093000CFFE824D022C09D1012F07D068463330FB
:100940004D2100222B1C00F0C3FE09E00CA83A2127
:1009500000222B1C00F0BCFE032CEFD1012FEDD0A8
:10096000784E2B1C301C5921002200F0B1FE734D33
:10097000042C01D1012F06D1684636305F210022B8
:100980002B1C00F0A5FE301C6C2100222B1C00F05B
:100990009FFE052C01D1012F06D168463930722106
:1009A0000022664B00F094FE0FA804210922664B3A
:1009B00003E0664804210022331C00F089FE00F0A9
:1009C000A3FD059B002B0AD0143B012B05D8052C59
:1009D00003D0962001F06AFD01E0FFF74DFD0320F2
:1009E000011CFFF7CDFC002000F00EFF0023051CCA
:1009F00006A905A806930593FFF782FC059B002B2B
:100A000074D007AD08AE281C311C09AA02F0E2FB25
:100A10000190002871D1281C02F0C6FC071C059823
:100A20001238052868D804F0AFFD0567240C670369
:100A3000601C00E0601D062104F05EFE00270C1C17
:100A40005BE0601E042804D804F09EFD060B0D1028
:100A50003A002B88013316E0A8780C2104F0ECFD55
:100A600019E001375FE0307801301BE07078013029
:100A700020E0601E042804D804F086FD0810121A35
:100A800022002B88013B2B80002445E0A8780C2114
:100A90000A3004F031FE0131A9703DE0013F42E02F
:100AA00030781730182104F027FE0422317040E01E
:100AB00070783B303C2104F01FFE0323717030E05E
:100AC0000023B370381C072104F016FE281C0A1CF2
:100AD0000991311C052C02D102F0D7FB02E0039BE7
:100AE00002F092FB01279623BB4008E0002D07D1BE
:100AF00001235F401F4003E0012796235B00029320
:100B0000059B842B17D0182B15D0029B029A013B12
:100B1000002A00D0D8E60EE0281C02F045FC052390
:100B2000071C0393CEE7381C291C02F06DFC02243D
:100B300005220392C6E713B0F0BDC046286100004D
:100B400071580000665800002061000073580000D2
:100B5000F7B502F0A1FA18200021FFF76DFC002480
:100B60006E4DFFF75FFC6E4EF8230022DB00F25063
:100B7000201C02F0B2FA002C02D00020012101E07A
:100B80000620032101F05EFC201C02F0A1FA01A95D
:100B9000071C6846002F03D0FFF704FC012729E05B
:100BA000FFF700FC009A002A24D1002CE0D15D4B15
:100BB0001B68002BDCD15A4B98331B68002B0BD1E0
:100BC000594BED18D4D500F049FC554B0022943315
:100BD0001A600224514DCBE7544B00941A6811322D
:100BE0001A60009A102AEBDC03F098FD009B013399
:100BF0000093F6E7002C0BD0009B182B01D0002FA0
:100C0000AFD000F089FC4A48FFF73CFC0123F366B3
:100C100000F032FF02F0AAF9009A182A64D1019F6D
:100C20000024F8B200F06EFDF823DB0001250194EA
:100C3000F550172846D00CD813282BD002D81128ED
:100C400019D04EE015282DD016284AD1FFF722FDE5
:100C50004AE026282ED004D819281ED0212811D0E9
:100C60003FE0442836D045283BD1E120000102F086
:100C700025FB281C32E02F4B1B68002B34D0FFF7DC
:100C8000EBFD05E02B4B1B68002B2DD0FFF710FE72
:100C9000009429E0FFF702FC26E0274B1868281A89
:100CA00001F010F80120FFF769FDFFF7E5FBFFF702
:100CB000A5FB19E0214B05221C70214B1A7000F096
:100CC00005FC11E01F4B1A6801321A60052A0BD18E
:100CD0001C6009E01C4802F0F1FA201CFFF76AFDD5
:100CE00002E000220197F250FFF764FB009801999F
:100CF00003F0F4FDF823DB00F358002B01D0FFF7DD
:100D0000BBFB074B94331B68002B03D100F0A6FB01
:100D1000012425E704F0B2FB21E7C04620BF020012
:100D2000D4040010680200100CFEFFFF94020010B3
:100D3000815800005001001008000010440100100C
:100D40000100001014010010F0F1FFFF73B5484DD1
:100D5000484B2A68484C9A4202D12C6001F050F866
:100D60002B68A34202D1424B00221A60434C02F08E
:100D70005FF800F00BFD4248002101F0DBF9002193
:100D8000404801F0D7F900F0D9FD00F079FF236861
:100D90000726B3432360236801252B4300202360EB
:100DA000021C0B2101F050F9201C374C102101F0DE
:100DB000C1F923680022B34323602368281C236001
:100DC000042101F041F9201C002101F0B3F901F0E8
:100DD00025F99620000201F09FFD2C4D01235B4276
:100DE00000202B60FFF7CAFC00232B605024012059
:100DF000FFF728FA00F044FF02F018F92B68002BE7
:100E000005D16420043C01F051FB142CEFD10020EB
:100E1000FFF7B4FC28211E4802F05CFB142001F00F
:100E200045FB1B48282102F055FB1A4801F05CFFE6
:100E3000192001F03BFB01F013FE002802D0FFF760
:100E40002DFB02E0013C002CF2DC02F0A1FB03F0E0
:100E500005FB1E2300930F2301930F480F49104AEF
:100E6000104B03F015FB104803F046FBFFF770FE34
:100E700008000010BE153E37E45BE1737440044087
:100E8000984004409C4004409440044050010010AD
:100E9000DE0300008B580000F9540000010300003D
:100EA000490700009402001080020010F7B50028E6
:100EB0003BD00378303B5A425341C0180378782B1B
:100EC00003D101301026012501E00A260025037810
:100ED000002201922D2B02D1012301300193002326
:100EE0000278002A1BD0171C303FFCB2092C02D814
:100EF0007343DB1911E020273A43002D08D0171C5B
:100F0000613FFFB2052F03D81B01573A134304E09A
:100F1000064801F0E9FE002007E00130E0E7019A11
:100F2000002A00D05B420B600120FEBD95580000F6
:100F30000378202B01D10130FAE77047031C303BC6
:100F4000DAB2092A01D8181C0AE020231843031C2E
:100F5000613BDBB2052B01D8573801E0012040424C
:100F6000704770B50E1CFFF7E3FF0025041C2078C6
:100F7000002807D0FFF7E2FF002803DB2D0105431F
:100F80000134F4E73560201C70BD000008B500F0A6
:100F900061FD011C014801F0A7FE08BDA358000037
:100FA00000B589B0684602F0E1F86946024801F0F0
:100FB0009BFE09B000BDC046DF580000F7B50F1C0E
:100FC00001A9161CFFF772FF002814D0019C0B49E1
:100FD000201C04F091FB0D1C081C642104F08CFB08
:100FE000281C3970642104F031FB04493070201C46
:100FF00004F02CFB01E001204042FEBD1027000060
:1010000037B50D1C48686A46694607310632FFF756
:10101000D5FF01AC69466A4620800132A8680231DA
:10102000FFF7CCFF6B4618702288044B9A4203D915
:10103000201C694602F029F937BDC0466B07000045
:1010400007B5486801A9FFF731FF019B3C205843D1
:1010500002F034F907BD000007235843054A101871
:101060009C30013B04D3C25C002AFAD0002000E08F
:1010700001207047D404001030B5194885B001F044
:1010800033FE0024651CA30719D1201CFFF7E4FFE1
:10109000002810D0281CFFF7DFFF00280BD0A01C71
:1010A000FFF7DAFF002806D0E01CFFF7D5FF002885
:1010B00001D004340EE00B48211C01F015FE211C68
:1010C000684602F079FA684601F0CCFE064801F065
:1010D0000BFE2C1CFF2CD5DD01F0D2FE05B030BD7F
:1010E0008A570000AF5800006FA1000070B50E1CB9
:1010F000FFF71EFF0D25041C0134631E1878FFF74F
:101100001DFF002806DB7055013DF5D2201CFFF7BE
:101110000FFF00E0002070BD70B5444C86B023681E
:101120000868251C002B06D1414801F0DDFD03F0C5
:1011300095F9012309E0012B0DD13E49082201F068
:1011400042FE002803D12368013323606BE03A4854
:1011500001F0CAFD5FE00378412B17D1374C023014
:10116000211CFFF7C3FF002855D00378422B52D132
:10117000211C02300E31FFF7B9FF00284BD0037855
:10118000432B48D1211C02301C3103E0532B06D1E4
:101190002B490230FFF7AAFF002844D13BE04D2B3A
:1011A0001FD1284C0230211CFFF7A0FF002832D0AD
:1011B00003784E2B2FD1211C02300E31FFF796FF02
:1011C000002828D00378472B25D1023001A9FFF74A
:1011D000C8FE019B002B1EDB184A1B4853651B49A8
:1011E0001DE001A9FFF7BDFE04782023061C9C43E7
:1011F00011D1301C02A9FFF779FF019B061CE118F1
:10120000FF2902DC02A802F0EDF9002E03D0013420
:10121000042CEED107E003F021F90B480C4901F052
:1012200063FD00232B6006B070BDC0465402001061
:10123000B85800008A570000CE580000D4040010AF
:101240001A050010FE040010DA580000F5570000DF
:10125000E458000037B54C682378002B25D0201CBB
:10126000FFF766FE01A9FFF77CFE019B041C002B23
:101270001BD0D8B2FF2B09DD00F060FA019B051CE2
:101280001812C0B200F05AFA019003E000F056FACA
:10129000002501900198002802D0291CFFF7CCF806
:1012A00023785A1E9341E418D6E737BD064A08B59D
:1012B000137801214B40137001D0044900E0044928
:1012C000044801F011FD08BD890300108858000092
:1012D000EB580000EF580000064A08B513780121CA
:1012E0004B40137001D0044900E00449044801F068
:1012F000FBFC08BD8803001088580000EB58000074
:10130000FE58000007B5486801A9FFF7CFFD019B13
:10131000002B01DC01230193019B1E2B01DD1E2309
:1013200001930199034A044B4A4304481A6001F0AF
:10133000DBFC07BD70170000840300100E5900008D
:1013400008B50C4A1378013BDBB21370002B0AD0AE
:10135000012B02D10849094A01E00949094A0A4812
:1013600001F0C2FC04E0094801F0BEFCFFF73EF9C1
:1013700008BDC0460000001032590000D8610000CE
:1013800036590000C16400003A5900005E5900005F
:1013900038B5051C002D09D0642402200021013C31
:1013A00000F078FE002CF8D1013DF3E738BD70B5B0
:1013B000061C01200821021C00F096FE07240120D3
:1013C0000821002200F090FE321C012522412A4013
:1013D0000020022100F088FE281C08212A1C00F0B1
:1013E00083FE013CEBD270BD10B50021041C0A1C29
:1013F000022000F079FE201CFFF7D9FF10BDF0B5E8
:10140000012385B002930023061C039372B60024C7
:1014100002AB1B59502040421843C0B2FFF7E4FF13
:101420000020FFF7E1FF1020FFF7DEFFE020FFF7CD
:10143000DBFF212767430025F71902200021012245
:1014400000F052FE785D0135FFF7B1FF842DF4D135
:101450000434082CDCD162B605B0F0BD08B5AC2070
:10146000FFF7C2FFAE20FFF7BFFFA520FFF7BCFFCD
:1014700008BD38B50122051C0C1C00F0E5FD281C38
:10148000211C012200F030FE38BD08B5AF20FFF767
:10149000ABFFA420FFF7A8FF08BD08B5AE20FFF7FB
:1014A000A3FF08BD10B5041CF820FFF79DFF201C0A
:1014B000FFF79AFF10BD10B5041C8120FFF794FFC1
:1014C0003F202040FFF790FF10BD000008B5074BFC
:1014D00020201B781843FFF787FF0A20FFF758FFEB
:1014E000034B1878FFF7E7FF08BDC0460100001066
:1014F0004401001008B5842202480021520001F086
:101500002DFC08BD8A03001008B50248FFF777FFDD
:1015100008BDC0468A03001008B501200821FFF766
:10152000A8FF00200221FFF7A4FF02200021FFF7FF
:10153000A0FF02200621FFF79CFF0320011CFFF7FC
:1015400098FF0320011C002200F0CEFD022006219E
:10155000002200F0C9FD06210122022000F0C4FD96
:10156000FFF7C8FFFFF7D0FFA220FFF73DFFA02045
:10157000FFF73AFFC020FFF737FF0020FFF792FF89
:101580000A20FFF705FF4020FFF72EFF2C20FFF772
:101590002BFF3220FFF7FCFE2E20FFF725FF322025
:1015A000FFF7F6FE2F20FFF71FFF0A20FFF7F0FEE0
:1015B000FFF78CFFFFF769FF08BD000083280ED8F6
:1015C0000F290CD8CB08842253430722C01811409E
:1015D000034B80220A41111C1A5C114319547047B5
:1015E0008A030010F7B55B18DBB20193019B9942A7
:1015F00015D28425CC086C4307270F408025041999
:101600003D41EFB2A618B44206DA054D65192B78B4
:1016100001343B432B70F6E70131C9B2E6E7F7BD71
:101620008A030010F0B51E1C87B00592F278049171
:101630005B68824201D2307845E0244AB478934214
:1016400005D10322041B54430192E4180CE0001B53
:101650000022824204DA1978013202315B18F8E77D
:101660001A789C1C5B780193A218002503922F1C0A
:10167000019B9F4226DA082200230292009373788E
:10168000009A9A421CDA029A082A06D1039B9C42CD
:1016900018D00022257802920134EB0708D5049A6D
:1016A000009BB818059AC0B29918C9B2FFF786FF17
:1016B000009B029A013301326D1000930292DEE723
:1016C0000137D5E7019807B0F0BDC0467959000051
:1016D000F7B5041C0D1C161C1F1C01F062FB201822
:1016E0000190019B9C420BD0832D09D82078291CA6
:1016F000321C3B1CFFF796FF01302D180134F0E738
:10170000F7BD000010B50021012204230A4C0C5D36
:10171000844203D118010243D0B20BE0013B002BFD
:1017200004D10132092A00DD1A1C042301312829C1
:10173000ECD1002010BDC046406100000F2302091B
:1017400018408000031F00D52833511E00200329B4
:1017500006D8242B04DC04218A1A0249CB18985C91
:101760007047C0464061000038B5051C0024054B99
:10177000291CE05C044B0134C01800F0DBFC0A2C8F
:10178000F5D138BD7C61000000400440F8B50D4F34
:101790003C68002C15D11020FFF7E6FF0A4B002211
:1017A000E65C1B195D78301C291C00F04DFC0234EE
:1017B000301C291C012200F097FC142CEED10123CF
:1017C0003B60F8BD480100106861000070B500245E
:1017D0000B4B0122E65C1B195D78301C291C00F0C4
:1017E00033FC0234301C291C002200F07DFC142C38
:1017F000EED10020FFF7B8FF024B00221A6070BD47
:10180000686100004801001038B5051CFFF7BEFFF5
:10181000002D09D007210122022000F015FC104BF9
:1018200080211A688A431A6000200B2100F032FCE4
:101830000124002805D000200B2100F02BFC44429D
:101840004441002D09D007210022022000F0FCFBBA
:10185000034B80211A680A431A60201C38BDC04619
:10186000FC3F0250F0B587B00026029001200391A2
:1018700004960596FFF7C8FFB04202D018230493E0
:1018800001260021284C009120786178012200F087
:10189000DBFB20786178002200F026FC234B9D1DA5
:1018A000012E24DC6A782F78111C381C019200F07C
:1018B000F1FB002808D100991D4AB3008A5C10335F
:1018C00069465A5001360BE02878697800F0E2FB4F
:1018D0000028F0D0381C019900F0DCFB0028EAD089
:1018E000009A144B0132023D00929D42D8D12778D4
:1018F0006578381C291C002200F0A6FB291C381C26
:10190000012200F0F1FB0C4902348C42BCD10020D2
:10191000864206D0049A029B05991A60039A012018
:10192000116007B0F0BDC04668610000386100007A
:1019300040610000366100007C61000008B50120B4
:10194000021C0B2100F080FB01200B21002200F083
:10195000CBFB03200221012200F076FB03200221B1
:10196000002200F0C1FB08BD234B37B51A681021D7
:101970008A431A60214B8022196892010A431A6037
:10198000051C0B210120002200F05EFB01200B2131
:10199000002200F0A9FB1A4B9F211A68194C8A43B8
:1019A0001A601A6818491A60184B186803F04EFE3E
:1019B0008023000218432A1C20600221032000F02B
:1019C00093FB142000F072FD2368FF2293432360F1
:1019D00023680F4A134323600E4B1B680193019B3E
:1019E000002BF9DA22680C4B13402360FFF7A6FFA7
:1019F00001980004800D3EBD388204408080044080
:101A00009840044000C0014000093D0098040010C7
:101A1000800000012CC00140FFFFFFF810B50C4C06
:101A20002068002813DA00202060FFF79DFF0A28B5
:101A30000ADC0120FFF798FF0138C023FF385B0064
:101A4000984201D801232360FFF778FF206810BD7A
:101A50000400001008B5FFF7E1FF002801D10020C5
:101A600007E00120FFF780FF011EF8D0014803F0D6
:101A7000EDFD08BD50BB120008B5FFF7CFFF0028F1
:101A80000AD0FFF7E7FFFA22031C0021C00FD200A3
:101A90009A424841014B186008BDC0464C010010F5
:101AA00008B5074B02221A60064BA2221960064BAA
:101AB0001A70A32258709A7000F008FE08BDC04644
:101AC000C4040010A0040010B404001008B5064BB4
:101AD00002311960054B00221A60054BA2221A70D0
:101AE000587000F0F3FD08BDC4040010A0040010FD
:101AF000B404001070B5051C0E1C0324281C311CF6
:101B0000FFF7CEFF0223FF33984202D0013C002CA6
:101B1000F4D170BD70B5051C0E1C0324281C311CAB
:101B2000FFF7D4FF0223FF33984202D0013C002C80
:101B3000F4D170BD0B4B10B51C6800239C420ED035
:101B4000094CA31CA270140A5C70140C120EDA70FB
:101B50009C70FFF7DFFF831EFF3B5A425341181C66
:101B600010BDC04650010010B404001070B50E4CFA
:101B700025680024A54215D00C4C160AA270E67008
:101B8000160C120E6271A371A21D26711C0A5470EC
:101B90001C0C1B0E9470D370FFF7BCFF841EFF3C1F
:101BA00063425C41201C70BD50010010B404001061
:101BB00008B5064B1A6800239A4205D0FFF79AFF32
:101BC000831EFF3B5A425341181C08BD50010010B0
:101BD00008B5074B00201B68834207D0022007216D
:101BE000FFF788FF0238FF384342584108BDC0461E
:101BF0005001001038B50F4B051C1B6800208342B4
:101C000017D00924641B631E062B10D8072C05D09F
:101C10000948A91E0918221C01F07EF8E8B2211C0F
:101C2000FFF778FF0238FF384342584101E00120B6
:101C3000404238BD50010010B6040010012010B51C
:101C4000011CFFF757FF0223FF3398420ED1094BC7
:101C500001211960084B1C78230709D0074B032288
:101C600022409A70081CFFF755FF01E001246442EE
:101C7000201C10BD50010010A4040010B40400107A
:101C800008B5FFF7DBFF02200121FFF733FF022336
:101C9000FF3398420FD1084B1B787F2B06D9842243
:101CA000022007215204054BFFF760FF09200421A1
:101CB000034AFFF73FFF08BDA4040010020114000F
:101CC0008080808010B500280CD0254B80211A68B8
:101CD0008A431A60234B1B68D907FBD5224B03228A
:101CE0001A6001E0204B1860204B012200211A608D
:101CF00019601A60196801221142FBD01C4B802127
:101D00001A601C4A49021468214311601A1C0028F9
:101D100004D1134B8024196821431960164B1968AC
:101D200088421CD01860002801D0144800E01448F4
:101D3000116803F03DFC134BFA2118608900041C64
:101D400003F084FC1E2358430F4BC821186049013F
:101D5000201C03F07BFC0D4B186001F053F810BD04
:101D6000388204400C800440708004407480044039
:101D7000788004408080044008000010006CDC0281
:101D8000001BB70098040010940400109C0400107D
:101D900008B500F04BF9134B00211A68120B12031F
:101DA0001A60114B1A68120B12031A600F4B1A6853
:101DB000120B12031A600E4B1A68120B12031A60F0
:101DC0000C4B012219600C4B1A6019601A601A68DA
:101DD00001200242FBD0094B23221A60FFF772FF59
:101DE00008BDC046008000500080015000800250B5
:101DF0000080035040800440448004400880044038
:101E0000014A024B1A60FEE70400FA050CED00E0FF
:101E100038B50F490F4800F067FF0F4D0024281C0C
:101E200000F062FF0D4A0E48A1581219D2682B1C0F
:101E3000143400F059FFF02CF4D10A4800F054FF9C
:101E400000F054FB011C084800F04EFF38BDC046AE
:101E50008A57000086610000D66100001C63000004
:101E600098610000A3610000C5610000F0B5404B1F
:101E70008BB01E68041C002E01D1351C0AE03D4BBE
:101E800002901B6801209B6802A998475EE03368B6
:101E90001E79019D2378002B31D0082D33D0237873
:101EA000202B01D10134FAE7002B28D06A1CAD00A9
:101EB00008356B460192EC50FF2E54D02278002A50
:101EC00007D0631C202A01D01C1CF7E700222270D7
:101ED0001C1C019A012ADCD1264E274B0D253360AC
:101EE000371C013D002D36D03B680298196800F080
:101EF0007BFF0028CBD03B6814333B60F1E7002D1B
:101F000024D0022D02D0B54206D911E003981B4916
:101F100000F06AFF0028F6D1164C19482368D968EA
:101F200000F0E2FE23681748196900F0DDFE0DE0BD
:101F3000104CE8B2236802A99B68984723689A6806
:101F4000114B9A4202D0114B03221A70084A1368AF
:101F5000002B0BD103E0281C291CFFF759FF0C486C
:101F600000F0C2FE02E0019D0026CAE70BB0F0BD02
:101F7000540200105C0200101C630000B757000000
:101F8000D2610000DF580000411300000000001083
:101F9000D961000038B5041C164D0A2808D002D8B3
:101FA000082811D01CE00D2802D07F280CD017E0A3
:101FB0002A6800231370104800F096FE0F4C201C76
:101FC000FFF754FF2C6013E00C4B2A689A420FD99C
:101FD0000B48211C00F088FE2B68013B2B6007E0BA
:101FE0000748211C00F080FE2B685A1C2A601C70D8
:101FF00038BDC04658020010D661000054010010E0
:10200000E561000008B500F02BFD002804D000F0C9
:10201000FDFCFFF7BFFFF6E708BD0000014A024BD9
:102020001A6070475401001058020010044B402100
:102030001A680A431A60034B01221A707047C0469F
:1020400080800440600200100F4B70B51B78061CA6
:102050000C1C151C002B01D1FFF7E8FF701E022895
:1020600003D80A4B8000C35800E0094B1A68012DC1
:1020700004D1A5402C1C14431C6003E00121A140A5
:102080008A431A6070BDC046600200100C640000F4
:102090000080005038B50F4B051C1B780C1C002B22
:1020A00001D1FFF7C3FF0020032D12D8281C012205
:1020B00003F06AFA02040608074B04E0074B02E04B
:1020C000074B00E0074B1B68A2401340181C421E40
:1020D000904138BD60020010FC3F0050FC3F0150B1
:1020E000FC3F0250FC3F03500F4B70B51B78061CA1
:1020F0000C1C151C002B01D1FFF798FF701E022845
:1021000003D80A4B8000C35800E0094B1A68012D20
:1021100004D1A5402C1C14431C6003E00121A14004
:102120008A431A6070BDC046600200101864000047
:10213000FC3F005038B5084B041C1B780D1C002BCD
:1021400001D1FFF773FF23681822934323602368AC
:102150001D43256038BDC04660020010054B3F227C
:102160001A60054B01221A60044B40211A688A4309
:102170001A60704724800440D880044038820440AC
:1021800008B5044B40211A688A431A60FFF7E6FF3E
:1021900008BDC0463882044008B500F05DFAFFF77C
:1021A00015FB0A480021FFF7C5FF09480021FFF78A
:1021B000C1FF08480021FFF7BDFF07480021FFF7D6
:1021C000B9FF06480021FFF7B5FF08BD08400440ED
:1021D00000400440AC400440144004401C40044013
:1021E00008B50120FEF72EF808BD000008B5124B17
:1021F0008022DA675200DA678022D200DA67802212
:102200005201DA6780221201DA6780229200DA67CF
:102210000A4A002313600121094A49421160094A10
:102220001360094A1360094A01231360084A1360C6
:10223000FFF7D6FF08BDC04604E100E00482044079
:102240000882044004C000403CC0004000C0004080
:102250000040014008B5064B1A6801321A60054B70
:102260001868FFF72FFDFFF7C1FFC046C04608BD45
:102270006402001008000010F7B5071C0C1C72B6B1
:10228000FFF78AFF524B1A68524B1A60002F01D099
:10229000514B00E0514B524A04211360514B524DB7
:1022A0001A680A431A6000232B60A1071ED04F4B07
:1022B0004F4A19680A401A6029684E4BA2070ED58A
:1022C000EC2252010A432A6080221A6052001A60EE
:1022D0008022D2001A60802252011A6003E080221C
:1022E00012010A432A60802212011A60002F53D083
:1022F000414B00241C60414B414E1C60414B301C43
:102300001C60414B211C1C60FFF714FF201C09219D
:10231000221CFFF799FE201C0921221CFFF7E4FE76
:102320003A4B80211A683A480A431A6033680722F8
:102330009343336033680222134333600A217843A6
:1023400003F036F9334B03221860334B1C60334BD8
:102350001A60334B334A19680A401A601A688021A0
:102360000A431A60234A8B001360204A11681943FC
:1023700011602A68022113432B602B4B01221A6043
:102380002A4B19602A4B1C491A601C601A60186895
:1023900001221042FBD00A60264B012252421A60F1
:1023A000254B00221B680193244B1A6062B630BF94
:1023B000C046214B019A1B689A4208D11F4B01224B
:1023C0001A601F4B1868FFF77DFCFFF70FFFF7BD82
:1023D0003882044034820440BF180000FF18000017
:1023E0003082044010ED00E004820440008204408A
:1023F0007FE2FFFF00E100E004C000400400014074
:102400006440044004400140048001408080044056
:10241000841E000018C0004008C0004014C00040E6
:102420003CC000400FF0FFFF788004407080044003
:1024300074800440088204406402001068020010A6
:102440000800001008B5FFF717FF08BD074B1A6812
:10245000013203D1064A1168013111601A68013254
:102460001A60044B1A6801321A6070477802001033
:10247000740200106C020010074B98420AD8074AF9
:1024800000231360064A01381060064A1360064BA9
:1024900007221A607047C046FFFFFF007802001055
:1024A00014E000E018E000E010E000E00B4A10B596
:1024B0001368002800D10120C1438B4208D911685C
:1024C000994209D3591C146809188C42FAD3F6E7CB
:1024D0001168C91A8142FBD310BDC04678020010B2
:1024E000014B18687047C04678020010064BFA216D
:1024F0001868064B10B589001C6803F059F8044BA6
:102500005C43201810BDC046780200107402001011
:1025100037894100034B01221A60034B1A680132CC
:102520001A60704700C000407C020010034B01227B
:102530001A60034B1A6801321A60704700000140AC
:1025400080020010002803D1044B01221A6003E02E
:10255000012801D1024B18607047C04604C00040FA
:1025600004000140002802D1044B186004E0012857
:1025700002D1034B00221A607047C04604C00040DD
:1025800004000140002801D1044B02E0012804D1DD
:10259000034B1A6802210A431A60704704C00040C6
:1025A0000400014010B5002900D1134900280DD1C5
:1025B000124B80241A6822431A60114B03221860C0
:1025C000104B1960104B1A60620211E0012811D102
:1025D0000A4B80221868520002431A600B4B0022FB
:1025E0001A600B4B032219600A4B1A608022920278
:1025F000094B1A6010BDC046FFFF000080800440F8
:102600007C02001018C0004014C00040800200107E
:10261000180001401400014000E100E08023102276
:10262000DB051A60094B08221A6000238022D205BC
:102630001268D10604D5064A934201D00133F5E76A
:10264000044898429B4158427047C04618000040D9
:10265000FF0F0000FE0F000008B58022154B12028C
:10266000DA67154B6C221A60144B154A1968002062
:102670001140196019681960124B19680A401A60F4
:102680001A6804211A600122FFF7DEFC00200421F1
:102690000122FFF729FD002005210122FFF7D4FCCC
:1026A000012200200521FFF71FFD074B00221A60C1
:1026B00008BDC04604E100E018000040304004407E
:1026C000F8FCFFFF3440044004800440F8B5174A8A
:1026D000174C002323601360164A202113608022C8
:1026E000D20511602168144A012903D0934203D016
:1026F0000133F7E7934203D1FFF790FF002014E086
:102700000E4F00253E68013E2368FF2B0CD83B6826
:102710009E4204D03E68FFF7E3FE051C0A35FFF732
:10272000DFFE8542F0D1E7E72068F8BD84020010A3
:10273000880200108C020010FF0F000090020010B1
:10274000034B01221A60034B1A6801321A6070476A
:102750000040014094020010174B70B501241C602A
:10276000164B1A6812191A60154B1A68002A22D0E3
:102770001A68144D013A1A601E68002E0DD02A689E
:10278000201C211CFFF7B0FC2B68201CE31A2B60D7
:102790002A680221FFF7A8FC0DE01B68201C2B60B3
:1027A0002A68211CFFF7A0FC2A68201C0221FFF7E1
:1027B0009BFC054B1E6070BD008001409C02001018
:1027C00098020010A002001004800140002803D1EC
:1027D000044B01221A6003E0012801D1024B18606A
:1027E0007047C0460440014004800140002802D1E7
:1027F000044B186004E0012802D1034B00221A6048
:102800007047C0460440014004800140002801D1C7
:10281000044B02E0012804D1034B1A6802210A4349
:102820001A607047044001400480014010B5002840
:102830000FD1124B80221C68920022431A60104B69
:10284000032218600F4B19600F4B1A608022D202CE
:1028500011E0012811D1094B80221868D2000243EF
:102860001A600A4B00221A60094B03221960094BB7
:102870001A6080221203084B1A6010BD8080044049
:102880009402001018400140144001409C020010C6
:10289000188001401480014000E100E008B5184BA9
:1028A0001A680E231340062B0DD1164B9E221B686F
:1028B000134205D0144ADBB25360144B1B681EE070
:1028C000D9071CD501E0042B05D1104B1868C0B204
:1028D00000F0B1F813E00C2B06D10B4B80225968A5
:1028E00052000A435A600AE0022B08D1054B1A68CD
:1028F000054B910601D5002200E001229A6008BD37
:102900000880004014800040A402001000800040B5
:1029100000487047A4020010F7B52D4B2D4C8022C3
:10292000002192030191061CDA67201C902200F01E
:1029300015FA019B0725A360274B284F1A68AA4365
:102940001A601968012211431960254B1968A943BF
:102950001960196811431960224B802118684901D8
:1029600001431960204B1A6083223A601F4A1268A3
:1029700019681F4B1868504302F01AFE311C0009F9
:1029800002F016FE1B4B10221B491A60030A0B6053
:102990001A4BC0B2032218603A60194A1560194AEE
:1029A0001D1C10680190106860230340602BFAD151
:1029B00010680123184202D02B680193F8E72370B6
:1029C0008022114B92031A6005230B60F7BDC046AD
:1029D00004E100E0A4020010A44004400C80004088
:1029E000A8400440808004409880044078800440DF
:1029F00098040010288000400480004000800040BF
:102A0000088000401480004000E100E008B5FFF7B6
:102A10007FFFC268031C1202120E8218D07BDA6894
:102A20001202120E0132D2B29A7352B2002A01DAA5
:102A300000229A7308BD10B5041CFFF769FFC26835
:102A40001204120E8218D473C2681204120E0132DC
:102A5000D2B2427352B2002A01DA0022427310BD90
:102A600008B5FFF755FFC268C36812021B041B0EAE
:102A7000120ED01A431E9841C0B208BD70B5002492
:102A80001D5D0619002D02D005550134F8E7121B13
:102A9000301C131C002B03DD0170013B0130F9E7F2
:102AA000D043C0170240A01870BDF7B5051C0191B6
:102AB0000093561E092B01D8041C0CE000980A2133
:102AC00002F076FD0199031C321C281CFFF7EDFF74
:102AD000071C2C1807E0671B002E04DD019B013E3C
:102AE00023700134F7E700980A2102F0A5FD303188
:102AF000781C2170FEBDF8B50C1CD9175F18051C99
:102B00004F40561E092F12D9381C0A21002B03DA18
:102B100002F04EFD434202E002F04AFD031C281C75
:102B2000211C321CFFF7E7FF041C2D1814E0002BBA
:102B300000DA961E2A1CA919891A002902DD1470D0
:102B40000132F8E7F443E41734402D19002B03DA7F
:102B50002D232B7001340135381C0A2102F06CFD45
:102B600030312970601CF8BDF7B5089F1E1C051C8C
:102B7000013A3B0901D1041C05E00093331CFFF727
:102B8000F3FF2C1806E0601B002A03DD2170013AD8
:102B90000134F8E70F231F40092F01D8303704E034
:102BA000002E01D0373700E0573727700130FEBDC7
:102BB000F0B585B0041C029101D000210170002500
:102BC0001178002906D1029F0023BD426CD22370E8
:102BD000281C6FE0029FBD42F5D2252902D00132A8
:102BE000217004E05178252904D121700232013589
:102BF0000134E5E7302902D0561C202100E0961C64
:102C000032782D3A50424241B618002230783027AF
:102C10007F423F18FFB2092F07D80A277A4382184C
:102C2000D2B2303AD2B20136F0E7AF18BC46029FBA
:102C3000BC4501D97A1BD2B2692818D00BD86328B9
:102C40002AD0642813D0582832D11F1D1B68201C9D
:102C5000009301231DE075280FD0782814D0732825
:102C600026D11F1D201C1B68FFF708FF0AE01F1D4F
:102C7000201C1B68FFF73FFF04E01F1D201C1B6882
:102C8000FFF713FF3B1C0BE01F1D1B68201C00936C
:102C90000023FFF769FFF5E718680433207001206F
:102CA000721C24182D188BE7013C2370681E01E06C
:102CB0000120404205B0F0BD10B50C1C131C64216E
:102CC000221CFFF775FF10BD00B5031C9BB00A1C4A
:102CD00001A8191CFFF7F0FF632800DDFEE701A83B
:102CE00000F0B6F81BB000BD0FB407B504A908C9C1
:102CF000181C0191FFF7E8FF03B008BC04B01847A7
:102D00000EB403B503AA08CA191C0192FFF7D4FF39
:102D100002B008BC03B0184730B50C1C04430323B1
:102D20002340041C002B01D0002310E0032AFBD910
:102D3000CC58C4500433D41A032CF9D8131F9B0861
:102D400001339B00C418C91803231A40ECE79342CF
:102D500003D0CD5CE5540133F9E730BD30B5031C39
:102D6000840701D1032A01D89A1814E00B060C0439
:102D70001D1C25430D430C022543031C20C384184E
:102D8000E41A032CFAD8131F9B0801339B00032479
:102D9000C3182240E8E7934202D019700133FAE7E2
:102DA00030BD021C031C981A0133591E09780029F2
:102DB000F9D17047031C0A781A70002A02D0013139
:102DC0000133F8E7704730B50023934208D0C45C64
:102DD000CD5C651B06D10133002CF6D1201C02E02E
:102DE000002000E0281C30BD10B50022835C8C5C04
:102DF000A34204D10132002BF8D1181C00E0181BAB
:102E000010BD000008B5094BFA211868890002F0CE
:102E10001DFCFFF731FB96200002FFF77DFD01202E
:102E2000FDF710FAFEF72CFF08BDC046980400100D
:102E300008B5FEF7ADFFFFF7F9F8FFF7A1F9FEF7C8
:102E40006BFBFEF757FBFFF7DDFFFFF7E7F808BD69
:102E500010B5041C2078002803D00134FDF742FA95
:102E6000F8E710BD38B5051C0E24013C04D3295DDC
:102E70000248FFF739FFF8E738BDC0462464000078
:102E800038B51948FFF730FF184C201CFFF7EAFF50
:102E9000174D4221281CFFF727FF201C0E30FFF79B
:102EA000E1FF4321281CFFF71FFF201C1C30FFF708
:102EB000D9FF1048FFF718FF201C4630FFF7D2FF5C
:102EC0000D48FFF711FF201C2A30FFF7CBFF281C0D
:102ED0004E21FFF709FF201C3830FFF7C3FF616D5B
:102EE0000648FFF701FF38BD27640000D404001036
:102EF0002D640000346400003A6400004064000067
:102F000003110A2253430F2210401818704738B596
:102F10000A21041C02F09AFB0A210501201C02F080
:102F2000EBFB281C084338BD08B5C12252000E2017
:102F30000221FEF7FFFD024B01225A7108BDC04677
:102F4000C804001010B5084C6379002B01D1FFF7BD
:102F5000EBFF23790C221A43A37901205B001A436B
:102F6000011CFEF7E7FD10BDC804001010B5074CAA
:102F70002379002B08D16379002B01D1FFF7D4FF0F
:102F800001232371FFF7DEFF10BDC046C804001007
:102F900008B5054B1A79002A05D000221A711A7259
:102FA000DA70FFF7CFFF08BDC804001010B501218B
:102FB0000220FEF7FDFD064B041C18787F23184005
:102FC000FFF79EFF034B5870DC71201C10BDC046FC
:102FD000A4040010C8040010014B01229A7070472D
:102FE000C8040010024B00229A701A727047C04643
:102FF000C804001008B5FFF7D9FF094B094A9978B2
:10300000002908D0197A012901D8013103E010689C
:103010000549086000E019720021D970116008BDEF
:10302000C80400106C0200107002001008B5FEF712
:1030300005FE0C23184003D0024B1A781043187079
:1030400008BDC046C804001010B5FFF7EFFF054BE0
:103050001A781C1C530701D5FFF7CCFF00232370FF
:1030600010BDC046C804001008B50020FEF7CCFB18
:10307000002801D0FFF7E8FF08BD000010B5054C9F
:103080000023E371FFF7F0FFE379002B01D1FFF795
:103090008DFF10BDC804001008B50948092102F0D1
:1030A00037FB084BFA22D2001A80FFF7E7FF064BE6
:1030B00000221A60FA22054B92001A6008BDC04631
:1030C000C8040010D20400106C020010700200103E
:1030D00008B5FFF7C9FF002008BD08B5FFF758FF86
:1030E00008BD000070B51D4C061C637822781B02D9
:1030F0001343A278A07912041343E2780D1C120640
:103100001343174A13401A0A237062701A0C1B0EDD
:10311000E3706379A27022791B021343114A1340B2
:1031200023711B0A6371FFF7EBFE0F4B1B88C0185E
:1031300030806079FFF7E4FEB070E078FFF7E0FEE2
:10314000F070A078FFF7DCFE28706078FFF7D8FEFB
:1031500068702078FFF7D4FEA87070BDA40400103A
:103160007F7F3F3F071F0000D2040010F0B58DB0F5
:10317000051CFEF72DFD002804D1281C1249FFF77D
:10318000BFFD1EE00AAE0BAC211C301CFFF7AAFFEE
:103190003388F7780793B378267808936378A47810
:1031A00009930A4B187900F0D7F8099B0490029311
:1031B000009701960394281C0549079A089BFFF77E
:1031C0009FFD0DB0F0BDC0464C640000A40400108B
:1031D0005164000070B5061C0D1C141CFEF7F8FCB1
:1031E00000280AD0301C291CFFF77CFF002C07D0D8
:1031F000044B00201B79236003E00120404200E0E3
:10320000201C70BDA4040010F7B504880E1C051C1A
:103210006421201C0092019302F00EFA114B8FB230
:10322000B078E41B1C80FFF772FE0F4CA070707822
:10323000FFF76DFEE0703078FFF769FE2071E878E7
:10324000FFF765FE009B6071A371A878FFF75FFE32
:10325000E071381CFFF75BFE20720198FEF7CAFC94
:10326000FEBDC046D2040010B404001008B502230D
:10327000FFF7CAFF08BD08B5021C501E824152016B
:1032800000200121FEF756FC08BD38B5041C0120C2
:103290000D1CFFF7F0FF201C00F086F8072102F05C
:1032A0002BFA201C0A1C291CFFF7E0FF9620400087
:1032B000FFF7FCF80020FFF7DEFF38BD73B5041CF4
:1032C000FFF774FE002801D100203BE01E4B5D7823
:1032D0001E1C7378AB4207D10A20FFF7E7F8FFF70F
:1032E00065FE0028F5D1EFE7FEF772FC0028EBD071
:1032F00001A96846FFF7F6FE684600F055F8051C80
:1033000001A800F031F8114B04199C420DD9E317C4
:1033100001221343ED18281C694600F075F8002CB3
:1033200001DA0B4B00E00B4BE418201C01A900F064
:1033300024F8281C072102F0DFF968460A1C01A9BD
:10334000FFF794FF76BDC046C80400107F5101000E
:103350008051010080AEFEFF07231840014B800022
:10336000C0587047C464000002783C235A43417837
:103370005218534382789818704738B50C1C3C217A
:10338000051C02F0B9F9281CA1703C2102F05EF97D
:103390003C2102F0B1F96170E121281C090102F021
:1033A00055F9207038BD000070B5837802210022E5
:1033B00099425241048896214901051C64180C2049
:1033C000A41A42439B18033B99205843052102301D
:1033D00002F03CF96E26FF3666436421A31086197D
:1033E0004942201CF61802F031F9C821361849006C
:1033F000201C02F02BF9034B3018C018EB78C018D2
:1034000070BDC046D382FFFFF8B5204B0C1CC51819
:103410001F4B8000C0181F4902F018F903235843BE
:10342000C617B60F3618B610AE19B600953E301C4A
:10343000194902F061F9CD17AD0F6D180527AD10D0
:103440007D430235281C992102F056F9081C391CCD
:1034500002F0FCF80130E0709921281C02F0F6F827
:103460000C21023002F048F94D1CEDB2A570301C61
:10347000094902F0EBF8094B0C21C6180E20401B3D
:1034800002F0E4F836182680F8BDC0467905000041
:10349000652F0400B13A0200B505000094EDFFFF6E
:1034A000012008B5011C021CFEF71EFE0120021CB3
:1034B0000221FEF719FE0120011C0022FEF7C4FDC7
:1034C000012002210022FEF7BFFD0120FFF78EF947
:1034D00008BD0000194B70B50D1C196807229143F7
:1034E00019601968012421431960154B061C1968DD
:1034F000201C914319601A68211C22431A60221C67
:10350000FEF7A2FD221C201C0221FEF79DFD0D4BA3
:10351000311C186802F09AF8011C201CFFF786F98C
:10352000201CFFF773F9084E201C3560FFF74EF999
:103530003368002BFCD1FFF7B3FF70BD7C40044023
:10354000804004409804001098020010F8238A017B
:10355000DB0013404A05920E1343F8221202114079
:1035600019430A23594330B5CA1083181C1CEB3485
:103570005D782478EA336C401B7824021C43835C1A
:10358000201C58400723194008418005800D30BD9C
:103590007047000008B5054B011E994201DD044B40
:1035A000C1180448EA38FFF7D1FF08BDFF17000033
:1035B00000F8FFFF006500000723594310B5084BD2
:1035C00059189C310023CC5C0F2222400270CA5C47
:1035D0000133120942700230072BF4D110BDC046EE
:1035E000D40400100723594310B5074B59189C31D8
:1035F00000234278047812012243CA540133023076
:10360000072BF6D110BDC046D404001070B5AC4CE9
:1036100086B0E36E6E465A1E934117363370A94B3F
:10362000E258D006400F0138062807D801F0ACFF59
:10363000040C2012181A1D00022509E0636E1633CF
:103640009B001B591D1C15E0636E16339B00E5584B
:1036500000230FE0A36DE56DAB420BDD0D2509E006
:10366000022503E00C25032304E00D252B1C01E0BB
:103670000D25EDE750111F2800D91BE101F08EFF49
:103680002000220029002C002F0033003B004400C2
:1036900048004C00540061006E00760083008F00EB
:1036A0009B00A800B800C500D500D300E100E400ED
:1036B000E700EF00FE0002010B010D010F011501F3
:1036C000E01801E0E0180E30EB1A591C02F020F867
:1036D000F0E0E0181C30F7E7211C0E3105E0E0189F
:1036E0000E30E1180BE0211C1C31201C1A1C2B1C75
:1036F00001F08DFADEE0E018E1181C300E31EB1A13
:103700005A1CFFF709FBD5E06F48011C0E31EDE7AD
:10371000E018011C1C31F2E7226E1021002A00D0B3
:103720000A21221C0E3206E0226E1021002A00D04F
:103730000A21221C1C32029100950196201C211C9A
:1037400053E0216E012232701022002900D00A229B
:10375000009501960292201C211C45E0226E10214A
:10376000002A00D00A21221C0E3213E0216E012211
:1037700032701022002900D00A2200950196029290
:10378000201C211C4DE0226E1021002A00D00A21AD
:10379000221C1C32009501960291201C6AE0226EC8
:1037A0001021002A00D00A21484A02910095019672
:1037B000101C111C19E0216E1020002900D00A20D5
:1037C000424A0290111C1C3900950196101C0CE015
:1037D000216E012232701022002900D00A223B49BA
:1037E000009501960292081C002201F01AFA61E08D
:1037F000226E1020002A00D00A20344A0290111CA8
:103800001C3900950196101C35E0216E01223270A2
:103810001022002900D00A222C490095019602921C
:10382000081C002227E001223270226E1021002A9B
:1038300000D00A21254A029100950196101C002112
:1038400019E0009620481BE00096204818E0226E00
:103850001021002A00D00A21221C1C3206E0226E10
:103860001021002A00D00A21221C0E320095019658
:1038700002910020211C01F0FCF91BE00096201CA5
:10388000002103E0211C1C310096201C1A1C2B1C5B
:1038900001F052FA0EE0201C02E00B4800E00B4859
:1038A000191C2A1C01F05FFA04E0201C191C2A1CB8
:1038B00001F063FA33780120E36606B070BDC046BC
:1038C000D4040010C4070000E2040010F00400104B
:1038D000064B10B51A1DD46F191C0831CC67D96F6F
:1038E000D1679A6F9867DA6710BDC046D40400109C
:1038F000064BD96F1A1D986F9967D16F08335967B6
:10390000D96FD1670022DA677047C046D40400102F
:10391000F8B5134C261C8C3630680130FFF73AFEA0
:10392000F923DB00E0500F4B0122E758A36E051C82
:1039300002409A4211D1830703D430680230FFF766
:10394000C7FFFF2292001540231CAD01BF108C332E
:103950002F431F60044B0122E2500220F8BDC046F5
:10396000D4040010C4070000AC0700000F4A104B3D
:1039700030B5D158131C8C331C68CB059B0E01202D
:103980008D0501D5403B02E0002B00D1031C8910BE
:103990000840916E884206D1111C8C31E3180B60EF
:1039A000044B0121D150012030BDC046D404001089
:1039B000C4070000AC07000008B5084B5A1CD07FB4
:1039C0009A1CD27F00011202104303331A7FDB7F5F
:1039D00010431B031843FFF77BFF08BDD4040010FE
:1039E00008B5FFF785FF0323044A0F219A18014009
:1039F000013311770011072BF6D108BDD404001054
:103A000008B5FFF775FF044B01211A1C8C321060BA
:103A1000024A995008BDC046D4040010AC0700000B
:103A200010B5064CA36E002B07D0FFF761FF231CD7
:103A30008C331860024B0122E25010BDD4040010F8
:103A4000AC07000010B5064CA36E002B07D1FFF7A2
:103A50004FFF231C8C331860024B0122E25010BD33
:103A6000D4040010AC07000008B5054A054B01213D
:103A7000D150054B1B68002B00D0984708BDC046AD
:103A8000D4040010BC0700003403001038B5154AF8
:103A9000154B00209850F822D2009A5882421AD032
:103AA000F622D200995881421ADD012909D1F72165
:103AB000C9005C58844204D00C4D58500A215C5116
:103AC00099509A58032A01DD0121D966F621013A5D
:103AD000C9005A5004E0064B1B68002B00D09847E1
:103AE00038BDC046BC070000D4040010B407000075
:103AF00034030010094BF822D2009A58002A04D04F
:103B0000F622D2009A58002A07DD054A0F219A585A
:103B10000133114099771211DA777047D4040010FD
:103B2000B4070000044B597F9A7F090112020A432F
:103B3000197F0A435A677047D40400100B1C093BD5
:103B400030B5012B0FD80023074A9C18257FC45C91
:103B5000A54205D0054B0839D0580143D15002E0A9
:103B600001330E2BF0D130BDD4040010A4070000A7
:103B700008B508290DD0192913D1427808231A4213
:103B800002D00022027002E00F230370072343706B
:103B900005E000230022C25401330E2BFAD1FFF7B7
:103BA00021FD08BD30B5114D85B06C6F002802D0E5
:103BB0000F239C4304436C67FF2C05DD281C1C303D
:103BC0000E2101F0A5FD0FE06846211CFFF7F4FC73
:103BD0006846211CFFF7CCFF00236846C15CEA1849
:103BE000013311770E2BF8D105B030BDD40400108D
:103BF000134B30B5596F0F229143041C0C4385B011
:103C00005C671D1C082C19D0FF2C17DC6846211C92
:103C1000FFF7D2FC6846211CFFF790FF0023EA184B
:103C2000127F6946CA5401330E2BF8D16846211C15
:103C3000FFF79EFF6846211CFFF7D4FC05B030BD9E
:103C4000D40400101FB50F4C616F082918D0FF294C
:103C500016DC6846FFF7B0FC6846616FFFF76EFF41
:103C60000023E218127F6946CA5401330E2BF8D1A3
:103C70006846616FFFF77CFF616F6846FFF7B2FC33
:103C80001FBDC046D404001010B50D4C631CD87F76
:103C9000A31CDB7F00011B021843E37F1843E31CD6
:103CA000DB7F1B031843FFF775FC0F23021C1A4030
:103CB00022770211134000126377A07710BDC0462F
:103CC000D4040010044B5A6E16329200D258121AC5
:103CD00051424A41DA667047D4040010044B5A6ED0
:103CE00016329200D158013900D50D21D1507047BC
:103CF000D4040010054B5A6E16329200D15801318F
:103D00000E2900D10021D1507047C046D4040010C4
:103D1000144B10B55A6E191C16329200D2580C2A48
:103D200005DC9A18507F117F0001021C17E00E4835
:103D3000F5241858A400A04205D00C4C2040B7240C
:103D4000A400A04207D18A18137F486D1B010211FD
:103D500013434B6505E09A18127F197F12010A433D
:103D60005A6510BDD4040010CC070000FFFEFFFF11
:103D7000264B10B55A6E16329200D2580C2A05D135
:103D800023495858F5218900884204D0FA21C900F6
:103D9000595800290DD0596D0F240C409A1808115C
:103DA000107754770901FF22114008431C775865AA
:103DB0002BE00C2A07DC596D9B180F220A400911D1
:103DC0001A77597721E0124AF5219A5889008A42D8
:103DD00005D010490A40B72189008A420DD15A6D99
:103DE0000F20191C1040293108701001FF210840D4
:103DF0001111021C0A435A6507E05A6D191C101173
:103E0000293108700F210A401A7710BDD404001020
:103E1000CC070000FFFEFFFF244B0F215A6E586DA8
:103E200016329200D258014070B500110C2A05D10B
:103E30001F4C1D59F524A400A54204D0FA24E40027
:103E40001C59002C09D09C18657F267F2D01354315
:103E50005D651D7F2077657726E00C2A08DC9C18BD
:103E6000657F267F2D0135435D65607721771CE0F6
:103E70000F4AF5249A58A400A24205D00D4C2240C6
:103E8000B724A400A24207D11A1C29321478117059
:103E900024012043586508E01A1C293214781D7F3C
:103EA00024012C435C651070197770BDD404001098
:103EB000CC070000FFFEFFFF08B503480E22011CDF
:103EC0001C39FEF729FF08BD0C05001008B5034892
:103ED0000E22011C1C31FEF71FFF08BDF00400106C
:103EE00008B504480022011C1C310D2300F08FFE90
:103EF00008BDC046F004001008B503480E22011C9E
:103F00000E39FEF709FF08BDFE04001008B503488E
:103F10000E22011C0E31FEF7FFFE08BDF00400105A
:103F200008B504480022011C0E310D2300F06FFE7D
:103F300008BDC046F00400100023044A00219A186E
:103F4000463201331170082BF7D17047D4040010AA
:103F5000C31C421E0020934207D004494000591858
:103F600046310978013B0843F5E77047D404001057
:103F700010B50B1D994208D0044A01248A18044048
:103F80004632147040100131F4E710BDD404001023
:103F900038B50020FFF7DCFF084C051C0021207F0E
:103FA000FFF7E6FF04202577FFF7D2FF0421051C69
:103FB000607FFFF7DDFF657738BDC046D404001091
:103FC00010B50020FFF7C4FF034C20770420FFF753
:103FD000BFFF607710BDC046D404001010B5054C7B
:103FE0000021207FFFF7C4FF607F0421FFF7C0FF9F
:103FF00010BDC046D404001010B50A4C231C8C33ED
:1040000018680130FFF7C6FAF923DB00E050021C04
:104010000F231A4022770211134000126377A07712
:1040200010BDC046D404001010B5084C0E21201C51
:1040300001F06EFB201C0E300E2101F069FB201CEC
:104040001C300E2101F064FB10BDC046D4040010EA
:10405000054B1A1C0E32197F187801330143D976AB
:104060009342F8D17047C046D4040010054B1A1C87
:104070000E32187F197801330140D9769342F8D176
:104080007047C046D404001030B5002185B00E4BF7
:10409000421C1818007F6C4608550D25D40F181CBB
:1040A000002395425C416442013122400E2901D037
:1040B000101CECE76C46E15CC218013311770E2B43
:1040C000F8D105B030BDC046D4040010074B10B580
:1040D0005A6E16329200D458611E1C19D1502077A6
:1040E000002901DA0D21D15010BDC046D4040010C2
:1040F000034A0023111C943198320B6013607047FF
:10410000D4040010034B0122943319684A401A600A
:104110007047C046D4040010074B0022191C8C3194
:104120000A601A67054A012199501A1C94321268D4
:1041300051424A41DA667047D4040010AC070000CF
:104140009A4B9B4910B5CC580F20A310994A1840A0
:10415000A411013812570E2844D801F015FA080EA0
:10416000151C20432643432D434343313500002A89
:1041700038DB8A184032002304E0002A32DB8A1838
:104180004032012393712BE0002A2BDB8A18403246
:104190009379CB6624E0201CFFF798FF20E0002AEB
:1041A00020DB101CFFF78EFD1AE0002A1ADB4B6E95
:1041B00016339B00CA5013E0201CFFF719FD0FE0D7
:1041C000201CFFF7EFFC0BE0002A0BDB101CFFF7B5
:1041D0005BFF05E00C2B20DD162B25D1FFF798FDAA
:1041E0000120E9E0982B02D100230B66F8E7982B19
:1041F00069DC382B02D101204866DDE0382B2EDC4B
:104200001C2B02D1FFF758FEEAE71C2B11DC0C2B0C
:10421000E0D1983101200860CEE00120002B00D1D0
:10422000CAE001204042C7E0182BFAD1FFF774FF23
:10423000D6E7282B02D100234B66D1E7282B04DCDC
:10424000262BEED1FFF794FDCAE72C2B02D1FFF706
:104250003DFEC5E7362BE4D1FFF7DEFDC0E7662B58
:1042600002D1FFF753FEBBE7662B16DC4C2B03D1C4
:10427000FFF7C2FE02209FE04C2B04DC3C2BD0D188
:10428000FFF72EFEACE7562B02D1FFF735FEA7E76E
:104290005C2BC6D1FFF790FBA2E76C2B02D1FFF796
:1042A0009FFB9DE76C2B04DC682BBAD1FFF7BCFEAB
:1042B00096E7762B02D1FFF733FE91E7882BB0D13A
:1042C000FFF718FC8CE7E62B02D1FFF779FE87E7B2
:1042D000E62B33DCC82B02D1FFF714FF80E7C82B95
:1042E00015DCA82B02D10120086665E0A82B04DCB0
:1042F0009C2B96D1FFF716FC72E7B82B02D1FFF783
:10430000F7FE6DE7BC2B8CD1FFF79CFC68E7D62B42
:1043100002D1FFF763FE63E7D62B04DCCC2B80D100
:10432000FFF7B2FC5CE7D82B02D1FFF779FB57E728
:10433000DC2B00D075E7FFF78BFE51E7F32B02D1A2
:10434000FFF7A4FB4CE7F32B17DCEC2B02D1FFF7B4
:104350008DFE45E7EC2B05DCE82B00D061E7FFF78D
:1043600071FB3DE7F12B02D1FFF7E6FD38E7F22BB9
:1043700000D056E7FFF778FB32E7F62B02D1FFF7C4
:1043800007FE2DE7F62B05DCF52B00D049E7FFF7FC
:10439000A5FC25E7F72B02D1FFF7ACFC20E7F82BB3
:1043A00000D03EE7FFF72CFB1AE7C046C407000029
:1043B000D404001000A1000010BDC04638B51E4C4A
:1043C0001E4D1F4B6159E150231C8C331868FFF7B9
:1043D000E1F8E26E1B4BA2660022E266E250032285
:1043E000605110401D1C022809D090420AD00128BB
:1043F00002D0FFF7A5FE07E0FFF78AFA04E0FFF717
:1044000005F901E0FFF7B2FA00280CDD6359002B33
:1044100004D1231C8C3319680A181A60231C9033AA
:1044200019680A181A60FA23DB00E258002A01D042
:10443000013AE25038BDC046D4040010C407000061
:10444000CC070000AC070000034B0122DA660F2204
:104450009A775A771A777047D404001070B5084CD1
:10446000F425ED006659201C064901F051F966510A
:10447000FFF7EAFF044A01236366A35470BDC046F8
:10448000D4040010D40700009C070000704700000F
:1044900030B50D4D049C28600C4801600C490A6041
:1044A0000C4A13600C4B039A1A600C4B0C4A1C60AC
:1044B000F423DB00D4500B4A0B4B1A600B4B0C4A15
:1044C00013600C4A136030BD6003001070030010CD
:1044D0007C030010440300103C0300101000001087
:1044E000D404001015460000340300108D44000071
:1044F0007403001058030010014B18607047C04649
:1045000040030010094B10B51A68191C084B002A0B
:1045100003D1084C2468226003E01A68904200DA54
:10452000101C186001230B6010BDC046480300102A
:104530006C03001040030010034B1B68002B01D1DB
:10454000024A13607047C04654030010480300102D
:10455000014B4A3318787047D404001070B5194DD8
:104560002B1C98331B68002B04D0174B1C680123AD
:104570001C4002E02B1C94331C68F523DB00EB5835
:104580009C4203D1114AAA58002A19D0002C02D10A
:10459000002B0BD114E00E4B0C4E1B68002B02D0ED
:1045A000201CA95998470023AB5106E0084B1B6813
:1045B000002B02D0201C211C9847F523DB00EC5077
:1045C00070BDC046D404001050030010A4070000C2
:1045D00060030010084B1860084B196000280AD0CF
:1045E000074A01231370074A00211170064A074940
:1045F0008850074A137070475C0300106403001072
:10460000780300104C030010B4070000D40400101D
:10461000380300102D4B73B51A682D4B11681868BC
:1046200081421BD000210091019112681A60294B30
:104630001B688B4202D0684601A99847264B009917
:104640001C68181C019A254BA14202D11C68A24289
:1046500002D0234C0125257001601A60214D224BA8
:10466000EB58002B10D01E490023CB56002B2CD02A
:104670001E4B00229A56012A27D100220A701C499B
:104680000A7002221A7020E0134B184C1868002898
:1046900007D00023E356002B03D1104B1968FFF716
:1046A00099FF0023E356124E022B04D1114A002336
:1046B0003370AB5023700023E356002B02D00A2046
:1046C000FFF720FF0023F356EB6673BD4403001091
:1046D0000C000010700300105C0300106403001055
:1046E0004C030010D4040010BC0700003803001075
:1046F00078030010B407000038B5064CF823DB003F
:10470000E358002B05D1E56E034AA350FFF782FF63
:10471000E56638BDD4040010BC07000008B5084A9F
:10472000084B126819688A1A05D5FA2252001A60D5
:10473000054B1A6801321A60FFF710FF08BDC0462A
:104740003C030010140000105003001037B5041C87
:104750000025002300930193124B1B68002B02D00D
:10476000684601A9984700980135002800D0002527
:104770000220FBF713FE0C4B1A680C4B11681868EB
:1047800081420AD012681A60FFF7C8FF002C04D0DB
:10479000013C002C01D1201C02E0032DD9DD0120B9
:1047A0003EBDC046700300104403001068030010B3
:1047B000F8B50E1C0E21041C171C00F0A9FF174BA6
:1047C00003259E4211DD092363730123237323E034
:1047D000301C0A2100F090FF301C61550A2100F0C6
:1047E00035FF0135061C0D2D01D0002EF0D1EF1B39
:1047F000033F27706B1E022B05D0E15C621BD218B1
:104800005173013BF7E70F235D1B013D6B1C032B2D
:1048100002DD00236355F8E7F8BDC046FFC99A3BA7
:104820000278002A01D1802252004378002B01D166
:1048300080235B00D01A7047F0B59B23234D5B00AB
:10484000EC5C85B003900E1C002C01D18024640028
:104850003023FF33EB5C002B01D180235B000293FC
:104860003823FF33EA5C80235B009C4203D00F2394
:10487000171C1F4000E007271548FFF7D1FF0299DA
:10488000421C631A802149000C1B0721C91B00949C
:10489000019103980F49FEF733FA00233370412446
:1048A000301CFEF77EFABA235B003718E818001BAD
:1048B000FFF7B6FF221C031C0749381C0134FEF722
:1048C0001FFA462CECD105B0F0BDC046D404001050
:1048D0000806001010A100001DA10000F0B5F7228D
:1048E000734CD200A150221C9432724B126895B0C6
:1048F000051C0E1CE050002A1AD118280BD1C32920
:1049000009D16D4B1B680F2B05D1201C38300E21AF
:10491000162200F067F967482058182806D1F723B7
:10492000DB00E358332B01D100F0F6F8FFF78CFDE4
:10493000F623DB00002D02D00A22E25000E0E55011
:10494000281C311CFFF746FE5C4D5D4E2B681B6832
:104950003360FFF7F1FD012323671E22002302923B
:104960000393584B1B68002B1AD0574D2B682F1CF4
:10497000002B15D01B68002B04D1544B1B689847A3
:104980003B68F7E72B681A68013A1A60504A1368C7
:10499000002B05DD013B1360002B01D1FFF7CCFD9F
:1049A000FFF70CFD002809DA231C8C331A6801324A
:1049B0001A60231C90331A6801321A60454B039821
:1049C000454D98420CD04023021C9A43434B9A42D7
:1049D00006D0434B984203D0F3239B00984211D159
:1049E0006359404A93420AD02022191C91433E4AFF
:1049F000914204D0402293433C4A934202D10A2080
:104A0000FFF780FD65593A4A0395251C8C352B68C4
:104A100093421BD0374A93420FD0374A934224D156
:104A2000FFF79CFDFBF7EAFC344B224A1860336821
:104A3000A050013B3360324B16E0324B1B68002B19
:104A400013D0314A0120A15898470EE02F4F3B6800
:104A5000002B0AD004A80CA9FFF7EEFE3B6804A8BF
:104A60000CA998472B6827332B60029D0298013DC3
:104A7000002813DC264B1E251B6898470F4B1A682D
:104A8000244B11681868814208D012681A60FFF739
:104A900033FEFFF743FE0D4B1B689847226F002A39
:104AA00001D002955DE7FFF759FD15B0F0BDC04696
:104AB000D4040010B40700001000001044030010DC
:104AC0000C00001048030010400300107403001095
:104AD0006C0300106E020000C407000026020000F4
:104AE0007A020000FB030000CB030000A3030000D8
:104AF0003E2700005C280000790D00005C030010D8
:104B00007E0D000060030010A40700007C0300106D
:104B10005803001068030010F7B52C4D00202B68D7
:104B20001C68FFF713FE2B681A689442FCD01B68C0
:104B3000274E2D33FF330193FFF786FC254CF623D8
:104B40000A22DB00E2501823A351F7231522DB00D1
:104B5000E250F8230127DB00E750231C90330022AA
:104B60001A60FFF771FC27672B68019A1B689A424D
:104B70000CD0FFF723FC2A68174B11681868814294
:104B8000F2D012681A60FFF7C9FDEDE7231C9033DD
:104B90001D68F823DF00012618200021E651FFF7E9
:104BA0009DFE0E4B281C196800F050FD0422011CCC
:104BB0000B48FFF7FDFD064818232350F72300227A
:104BC000DB00E651281CE250FEBDC0464403001045
:104BD000B4070000D4040010680300103C03001068
:104BE0000C05001070B5002A10DD047801231C406C
:104BF0004B1E002B08DBC55CE4006E083443C45434
:104C00000124013B2C40F4E7013AECE770BD30B5DC
:104C10009A4205DC845C8D5C85548C540132F7E744
:104C200030BDF0B5069E051C07A804783078002A30
:104C300017D0059EB34217DCCE5CD75CF7193F183E
:104C40000020A74201DB3F1B0120EF540133F0E7B6
:104C5000CA5C12180020A24201DB121B0120EA5498
:104C60000133059A9342F3DD01231840069B187027
:104C7000F0BDF7B50AAC2478099D0094089E2C7805
:104C8000002833D000292ED0002A1CD0B3424EDC9D
:104C9000CF5CD55C7F1B3F1B0024A74204DA009C3D
:104CA0003F190F2427400124C7540133EEE7CA5CA3
:104CB000121B0024551C04D1009C0F22013C2240F1
:104CC0000124C2540133B342F1DD30E0D15C4942EA
:104CD000091B0024A14204D0009F0F24C9192140C0
:104CE0000124C1540133B342F0DD20E0002914D087
:104CF000002A08D0B3421ADCCD5CD05C0133281AFC
:104D0000041BE40FF6E7B34211DCCA5C0133141B49
:104D1000013462425441E4B2F5E7B34207DCD15CAE
:104D2000013349420C1B611E8C41E4B2F5E70123BB
:104D30001C40099B1C70F7BD70B5049C01252570B3
:104D400000290BD09A420BDC865C8D5CAE4209D107
:104D50000132F7E7815C002904D101329A42F9DD82
:104D60000023237070BD914204DA43185B784354EA
:104D70000131F8E70023435470478A4205DD831868
:104D8000013B1B788354013AF7E7002383547047B3
:104D9000F7B5134A134C13785278C35C134000D014
:104DA0004023114923601231009100220023A618EC
:104DB0007360009B0125123B1F785978C75D39420B
:104DC00002D077682F437760009F02336D00BB42AB
:104DD000F2D1123304320093282AE7D10020FEBD1D
:104DE00004010010380E001050000010122330B5DE
:104DF0004B43334A0131D318052251431A785C786A
:104E0000825C144204D02F4A5F245218947054706C
:104E10009A78DC78825C144204D02A4A7C245218A6
:104E2000533214701A795C79825C144204D0254A9A
:104E30007C245218A33214709A79DC79825C144273
:104E400007D0204C5F226418251CA235A1342A709B
:104E500022701A7A5C7A825C144204D0194A7C244B
:104E60005218A03214709A7ADC7A825C144204D010
:104E7000144A7C245218503214701A7B5C7B825C7A
:104E8000144207D00F4C5F226418251C5235513450
:104E90002A7022709A7BDC7B825C144204D0094A1F
:104EA0002E245218A43214701A7C5B7C825C13424C
:104EB00004D0044B5918F43127230B70002030BD67
:104EC00050000010A80C0010F8B52E4D061C00274D
:104ED0002C1C281C20214F22FDF740FF002F04D05E
:104EE0002A1C7C2339322B7013702B1C4F33002269
:104EF00001371A705035052FEBD1211C2D23383185
:104F00000B70211C37310B70A121A3706370490015
:104F10005F2363544221FF316354A321490062544B
:104F2000194A11785278715C0A4204D0221C53321B
:104F30005234137023700024211C301C0134FFF7FD
:104F400055FF0A2CF8D10024104B114DE25C1B19BF
:104F5000B15C58780F4A6300084201D0D15805E08F
:104F6000D058FDF71EFF0C49091A0A31281C0234DB
:104F700000F0D8FB122CE7D1281C084900F0D2FB26
:104F80000520F8BDA80C0010040100101800001046
:104F9000E80D00102C0000100601001025A10000F3
:104FA000F0B5944B87B003901F68FCF7A3FA9249C1
:104FB0000022924C02910192019B0C255D43002B33
:104FC00000D101258B4B1968032903D0042900D196
:104FD0003EE202E0884A029202E0022900DCAAE0F6
:104FE000002305AA537023687F2003405B2B72D0F7
:104FF0002CDC232B00D19AE014DC062B50D006DCED
:10500000002B4BD0022B00D094E0492390E01C2BC6
:1050100000D18AE0212B00D185E0072B00D089E068
:10502000372385E0402B6ED008DC392B6FD03F2B27
:1050300067D0382B00D07DE04C2379E0502B72D024
:10504000542B74D04F2B75D1332371E0732B68D060
:1050500012DC662B41D007DC5E2B5AD0622B64D069
:105060005C2B67D14F2363E06F2B3CD0712B54D066
:105070006D2B5FD135235BE0792B4CD006DC762B92
:105080004DD0772B41D0742B54D148E07D2B26D0C6
:105090007F2B26D07C2B4DD1422349E0202347E0B3
:1050A00031231370019B022B00DCB8E1231C083B69
:1050B0001B680340542B0AD00199032900D1AEE1AB
:1050C000231C0C3B1B681840542800D0A7E14C223D
:1050D00005AB1A70A3E132232AE0342328E03623FB
:1050E00026E0382324E039231370019B062B00DCD3
:1050F00095E1231F1B6818404723232800D08EE129
:1051000016E0302314E02D2312E0412310E0432366
:105110000EE044230CE045230AE0462308E0482340
:1051200006E0502304E0522302E0552300E04E2322
:10513000137074E1CF1E012F62D0022F00D1E1E085
:10514000002F00D03EE1226801231A4205D0A81C9E
:10515000C0B2391C0522FCF745FA23689B0706D527
:10516000E81D0121C0B20A1C0323FCF73BFA2168A9
:105170000423194205D0E81DC0B205210122FCF725
:1051800031FA2268120706D5A81CC0B209210522EF
:105190000123FCF727FA2368DB0606D5681CC0B29A
:1051A000052101220423FCF71DFA2168890606D592
:1051B000681C0121C0B20A1C0323FCF713FA226801
:1051C000520606D5A81CC0B2042105220123FCF713
:1051D00009FA23681B0607D5281C0930C0B209212B
:1051E00002220123FCF7FEF92168C90500D4E9E099
:1051F000DCE0C0461401001028610000380E0010E9
:1052000022683A420ED0EEB2B01CC0B20021052294
:105210003B1C0336FCF7E6F9F0B2391C03223B1CB9
:10522000FCF7E0F923680222134205D0A81DC0B2A2
:1052300001210323FCF7D6F921680423194205D084
:10524000A81DC0B205210222FCF7CCF9226808266D
:10525000324211D0EBB2181C02300093C0B20921C7
:1052600005220123FCF7BEF9009B311C0333D8B2A1
:1052700003220123FCF7B6F92168C90606D5681C8C
:10528000C0B2052102220423FCF7ACF92268920681
:1052900006D5681CC0B2012102220323FCF7A2F943
:1052A00023685B060ED5EEB2B01CC0B20421052205
:1052B00001230336FCF796F9F0B2052103220123FE
:1052C000FCF790F92168090607D5281C093002224D
:1052D000C0B20821131CFCF785F92268D20571D5EC
:1052E000EDB22E1C0A36F6B2301C0821022203232E
:1052F000FCF778F90935301C0B21FCF75FF9E8B2AF
:105300000B215DE02368DB0706D5681CC0B20021D5
:1053100007223B1CFCF766F921680222114205D0E6
:10532000A81DC0B200210623FCF75CF92268042105
:105330000A4205D0A81DC0B202220623FCF752F98A
:10534000236808210B4205D0681CC0B20722022343
:10535000FCF748F92168C90606D5681CC0B20421CB
:1053600002220623FCF73EF92268920606D5681C45
:10537000C0B2002102220623FCF734F923685B0641
:1053800006D5681CC0B2042107220223FCF72AF9C3
:105390002168090607D5281C09300222C0B208215D
:1053A000131CFCF71FF92268D2050BD5EDB2281C9F
:1053B0000930C0B20B210A35FCF700F9E8B20A2126
:1053C000FCF7FCF8019B0434013301930B2B00D054
:1053D000F2E5214B1B68002B05D020480021092253
:1053E0001F4BFCF775F91F4D00240235AB1E1A78D0
:1053F00003996B1E8A5C1B78134208D01A4BA200DB
:10540000D0581A4B0922E15C154BFCF761F90134C5
:105410000235092CEAD1FCF777F807B0F0BD00227D
:1054200005A8291C029BFCF753F92268120605D532
:10543000E91D0F480022029BFCF74AF92168C905C3
:10544000C0D5E91D0B480022029BFCF741F9B9E7E2
:10545000094B0293C4E5C0464C0100102FA1000087
:1054600020610000180000101801001086A1000043
:10547000116200002DA100003061000038B5FFF777
:1054800067F80624002805D1FCF73EF838BD013442
:105490000E2CF9DC0321201C00F0D8F80321C5B242
:1054A000201C00F029F9281CC9B2FCF787F8092C48
:1054B000EDD10B24EEE7000038B5041CFFF768FCC3
:1054C000201CFFF76DFD094B1B78002B0DD0201C15
:1054D000FFF7FAFC064CC8235B00E518211C0548C1
:1054E0005034FDF701FCAC42F8D138BD89030010FF
:1054F000A80C0010DF58000000B589B000280ED0BD
:10550000FBF7C3FF01A80921FEF756F868461230E1
:105510000A21FEF751F801A8FFF7CEFF08E0FBF7DC
:10552000BCFF044B1B78002B02D00348FDF7DCFBCB
:1055300009B000BD8903001031A10000FEE7FEE7BD
:1055400008B500230B4A0C499A188A4204D20B4929
:10555000C95C01331170F5E7094B0A4A591C013B3C
:10556000934203D200221A700B1CF6E7FBF7EEFB06
:10557000FEE7C046000000103C0100108FA10000B3
:105580003D010010640E001002B471464908490044
:10559000095C49008E4402BC7047C04603B47146A2
:1055A000490840004900095A49008E4403BC70472D
:1055B000002934D00123002210B488422CD30124C6
:1055C0002407A14204D2814202D209011B01F8E75B
:1055D000E400A14204D2814202D249005B00F8E714
:1055E000884201D3401A1A434C08A04202D3001B40
:1055F0005C0822438C08A04202D3001B9C08224373
:10560000CC08A04202D3001BDC082243002803D0B0
:105610001B0901D00909E3E7101C10BC70470028E2
:1056200001D00020C04307B4024802A140180290F4
:1056300003BDC046D90000000029F0D003B5FFF734
:10564000B9FF0EBC4243891A1847C046002941D011
:1056500010B4041C4C40A44601230022002900D5AC
:105660004942002800D5404288422CD30124240717
:10567000A14204D2814202D209011B01F8E7E400F1
:10568000A14204D2814202D249005B00F8E788427D
:1056900001D3401A1A434C08A04202D3001B5C08F5
:1056A00022438C08A04202D3001B9C082243CC0852
:1056B000A04202D3001BDC082243002803D01B09B0
:1056C00001D00909E3E7101C6446002C00D54042D4
:1056D00010BC7047002806D003DB0020C043400800
:1056E00001E08020000607B4024802A140180290A1
:1056F00003BDC046190000000029EBD003B5FFF739
:10570000A7FF0EBC4243891A1847C0467047C046DF
:1057100042180023002903D0037001309042FBD1CE
:105720007047C04670B5061CB30717D133680F48E1
:105730000F4D1A189A43301C2A420FD104300268C8
:105740000A4BD41894432C4208D104300268074B0A
:10575000D41894432C42F1D000E001300278002AA2
:10576000FBD1FDF727FB301C70BDC046FFFEFEFEDF
:10577000808080805B4025303278253032785D0D26
:105780000A0025732025730D0A00444D31355F4D05
:1057900031420053455249414C20434F4E534F4CE8
:1057A00045007265616479000D0A4279652E2E2EDE
:1057B0000D0A004E4F00203F002573202573202046
:1057C00025694D485A0056333100202025692E2581
:1057D000303369560020257352544320005245410E
:1057E000445920464F5220464C415348494E4700A9
:1057F000444D3431204F4B00424144204B45592009
:105800002530327800202D2025303278004C43445A
:105810003A25303269202D202569005052455353D6
:1058200020454E54455220544F2053415645005375
:10583000574953534D4943524F532028432920324F
:105840003031302D323032300053495A453A2569D3
:1058500020555345443A256920465245453A256925
:1058600000535441434B3A0025633120484F555271
:10587000002D005254432052454144204641494C9A
:10588000007475726E6564206F6E003C524553451E
:10589000543E0D0A00426164206E756D6265722E81
:1058A0000D0A004241543A2025696D560D0A000D3B
:1058B0000A2530327820200057616974696E6720AC
:1058C000666F7220646174612E2E2E0D0A00426193
:1058D00064206D6F64656C0D0A005265616420255B
:1058E000730D0A004641494C4544006F6666004C02
:1058F00043442064656275672025730D0A004B429E
:1059000044206F75747075742025730D0A00436F01
:105910006E736F6C652074696D656F757420736547
:105920007420746F202569206D696E757465730D20
:105930000A006F6E650074776F0053617920626FA3
:105940006F746C6F61646572202573206D6F726572
:105950002074696D652573202E2E2E0D0A004C6172
:10596000756E6368696E6720626F6F746C6F6164D7
:105970006572202E2E2E0D0A00000000005C000C27
:10598000000C7C287C7C447C241048285408000CA3
:1059900000384400443800201008103810804000BF
:1059A000101010004000201008384438007C0064BB
:1059B00054484454281C107C4C54243854200474FB
:1059C0000C285428085438005000805000102844F7
:1059D000282828442810045408384C5C7814787C13
:1059E00054283844447C44387C54447C140438445F
:1059F000347C107C007C0020403C7C106C7C40405F
:105A00007C087C7C047C7C447C7C14083844787C56
:105A10001468485424047C047C407C3C403C7C203A
:105A20007C6C106C1C601C64544C7C44000810207E
:105A3000447C0008040880808004080078447800D2
:105A400007080400000000BF01BF010905000007AE
:105A5000000700070007130A00002000E400FC0014
:105A60003F00E700FC003F002700040F0800000C87
:105A7000011E01FF03FF032201E201C2190D000014
:105A80000E001F0011019101FF007E00FC00FE01CD
:105A900013011101F001E0140A0000EE00FF0111F2
:105AA000011101BF01EE00E001300110010503000A
:105AB000000F000F0A050000F800FE0307070104AD
:105AC0000B060000000001040707FE03F80F0800A2
:105AD0000000000A000E001F001F000E000A11093E
:105AE0000000100010001000FE00FE00100010006A
:105AF00010080400000004800780030D0700001058
:105B00000010001000100010001008040000000039
:105B1000800180010D07000C000FC003F0003C0065
:105B20000F00030F080000FE00FF01010101010149
:105B300001FF01FE10080000000002010201FF0148
:105B4000FF0100010001100800008601C70161018A
:105B5000210131011F010E010F08000082008301A5
:105B6000110111011101FF01EE110900003000388F
:105B7000002C002600FF01FF012000200F0800007C
:105B800080009F011F0111011101F101E10F0800C7
:105B900000FC00FE010B0109010901F901F00F08E9
:105BA000000001000100C101F1013D000F00030FE1
:105BB000080000EE00FF01110111011101FF01EECB
:105BC0000F0800001E003F0121012101A101FF007B
:105BD0007E0804000000008C018C01080400000015
:105BE000048C078C0312090000200070005000D8BC
:105BF0000088008C010401040111090000480048DC
:105C000000480048004800480048004811090000CA
:105C1000040104018C018800D80050007000200DA0
:105C200007000002000300B101B9010F0006190DC1
:105C30000000F800FC010603FB06FD05050505054F
:105C4000FD05FF050601FC01F8120900008001F0C6
:105C5000017C004F004F007C00F00180010F080024
:105C600000FF01FF01110111011F01FE01E01109F7
:105C700000007C00FE00830101010101010183019C
:105C80008211090000FF01FF0101010101010183EF
:105C900001FE007C10080000FF01FF01110111014D
:105CA0001101110111010F080000FF01FF01110096
:105CB00011001100110001120900007C00FE008398
:105CC00001010121012101E301E20112090000FFAC
:105CD00001FF011000100010001000FF01FF010A79
:105CE0000500000101FF01FF0101010B0600010099
:105CF0000101010101FF01FF10080000FF01FF0188
:105D000038006C00C6008301010110080000FF018B
:105D1000FF0100010001000100010001160B00005D
:105D2000FF01FF010F003C00F000F0003C000F00FD
:105D3000FF01FF0112090000FF01FF010F001C001D
:105D40007000E001FF01FF01130A00007C00FE006B
:105D500083010101010101018301FE007C0F0800A4
:105D600000FF01FF012100210021003F001E140A55
:105D700000007C00FE008301010101010103830793
:105D8000FE047C0412090000FF01FF012100210034
:105D90007100DF008E010001110900008E009F01DB
:105DA0001101110111011101F301E21109000001BA
:105DB0000001000100FF01FF0101000100011109C4
:105DC00000007F00FF008001000100018001FF0052
:105DD0007F1109000007001F007800E001E0017852
:105DE000001F0007190D00000F007F00F001E00107
:105DF0007C001F001F007C00E001F0017F000F12FB
:105E00000900008301C7016C00380038006C00C72E
:105E100001830111090000010007001E00F801F8CC
:105E2000011E00070001120900008101C10161018A
:105E3000310119010D0107010301000404020000F2
:105E40007F0109050000070000000000070B064461
:105E500000FF0144004400FF01440B0600008C00D9
:105E60001201FF032201C40D0782004500250092A4
:105E70000048014401820C060000E60019012601D9
:105E8000C000200107040000000001000208040017
:105E9000000000FE0101020804000000000102FEF3
:105EA000010B0600008800500020005000880B06FF
:105EB000000020002000F800200020060300000061
:105EC0000400020B0600002000200020002000201B
:105ED00006030000000000010905000080016000C9
:105EE0001800060B060000FE00010101010101FE81
:105EF0000804000002000200FF010C0600008201FD
:105F00004101210111010E010B0600008200010177
:105F100011011101EE0B060000600058004600FF61
:105F200001400B0600009F00090109010901F10B66
:105F3000060000FE00110111011101E20B06000034
:105F40000100C10131000D00030B060000EE00113D
:105F50000111011101EE0B0600008E00110111016B
:105F60001101FE0804000000008C018C01080400EF
:105F7000000000000208010A05000020005000880F
:105F80000004010B0600005000500050005000506B
:105F900009050000040188005000200B06000002E3
:105FA000000100610111000E0D0778008601320129
:105FB0004902390242027C0E07800170004C004306
:105FC000004C00700080010B060000FF0111011160
:105FD000011101EE0B06FE000101010101010101A9
:105FE000820B06FF0101010101010182007C0C0608
:105FF0000000FF0111011101110101010B06000058
:10600000FF01110011001100010C06FE0001010149
:106010000111019100F2010C06FF011000100010A7
:10602000001000FF010804000000000000FF01074D
:1060300004C00000010001FF0E070000FF0118006E
:1060400024004200810000010C060000FF01000155
:106050000001000100010E07FF010C003000C0002C
:1060600030000C00FF010C06FF01060018002000A4
:10607000C000FF010B06FE00010101010101010149
:10608000FE0B06FF0111001100110011000E0C069D
:10609000FE000101010141018101FE020C06FF0128
:1060A0001100110011002900C6010B0600008E002E
:1060B000110111011101E20B06000001000100FFB6
:1060C000010100010B06FF000001000100010001B9
:1060D000FF0D0703001C006000800160001C00032E
:1060E0000D071F00600080017C00800160001F0E12
:1060F0000783014400280010002800440083010D9C
:1061000007030004000800F00108000400030E0764
:106110008101410121011101090105010301000073
:1061200003072061795900000D0C205A3A5E0000E7
:106130000D0C205A3F5A000000070008000A010019
:10614000181110133831303378717073C8C1C0C35F
:106150008881808384848782C5C4C7C2757477723E
:1061600035343732151417120207020802010003F2
:106170000109030402040205030500062024282C5B
:10618000383C4044484C4669726D77617265202501
:10619000735F5633310D0A00252D3130732025737E
:1061A0002573000D0A5479706520273C636F6D6D6F
:1061B000616E643E203F2720666F722070617261BD
:1061C0006D730D0A00557074696D65202575730D2A
:1061D0000A0025730D0A0D0A00564F5941474552D2
:1061E000203E3E200025630048656C70004E6F2005
:1061F000706172616D73004B6579207072657373A5
:10620000003C6B6579313E203C6B6579323E202E37
:106210002E2E0044756D70206D656D6F7279004C87
:106220006F6164206D656D6F727900637400436FF8
:106230006E736F6C652074696D656F7574003C6D6D
:10624000696E757465733E00626F6F746C6F616424
:10625000657200496E766F6B6520426F6F746C6F6C
:106260006164657200536179207468726565207499
:10627000696D6573004765742074696D650074739A
:10628000005365742074696D65003C595959594D26
:106290004D44443E203C48484D4D53533E007464A9
:1062A000005570646174652074696D65003C6F66AB
:1062B000667365745F696E5F6D696E757465733E54
:1062C000006B6200546F67676C65206B6579626F65
:1062D000617264206F757470757420746F20636FC1
:1062E0006E736F6C6500546F67676C6520646973CB
:1062F000706C6179206F757470757420746F206391
:106300006F6E736F6C6500526561642062617474B6
:1063100065727920766F6C7461676500B75700000D
:1063200000000000111E0000E8610000ED610000A7
:10633000EB610000FF00000055120000F761000053
:1063400001620000C164000000000000791000003C
:1063500013620000ED6100004F64000000000000C7
:10636000191100001F620000ED6100002B620000A7
:1063700001000000051300002E6200003E620000D4
:10638000486200000000000041130000536200005A
:10639000656200002C62000000000000A10F0000F8
:1063A00075620000ED6100007E62000002000000E6
:1063B00001100000816200008A6200009E620000FD
:1063C0000100000041100000A1620000AD62000069
:1063D000C162000000000000D9120000C462000089
:1063E000ED6100009F62000000000000AD1200009F
:1063F000E6620000ED610000C262000000000000E3
:106400008D0F000007630000ED6100000080015067
:106410000080025000800350FC3F0150FC3F0250BE
:10642000FC3F03502578000D0A413A20002020252A
:10643000633A20000D0A533A20000D0A4D3A20001D
:106440002020473A20253032780D0A006661696CB9
:1064500000253034692D253032692D2530326920F0
:10646000253032693A253032693A253032692025A3
:106470007300253032783A253032783A2530326947
:106480002E253032690025303278203A20256920C7
:106490002569203A2025303278004E4F205254434F
:1064A00000253032783A253032783A25303278007B
:1064B000253034782D253032782D25303278202043
:1064C00025730000E4640000E8640000EC64000050
:1064D000F0640000F4640000F8640000FC64000054
:1064E000D86100004D4F4E005455450057454400BB
:1064F00054485500465249005341540053554E00EC
:10650000CCC5ED2D1207EE76A609CFA6C6FC205FFE
:10651000FD8D1416A5B8757A3E3979BAAC30388E2F
:106520004526943C71EA4D1DFC6918F8374D202D25
:106530005431210C7B81EFB98C658A36C3DF9BAF68
:106540001E308AD6E807680B0BE035688B58BB36DF
:106550007E32A97A0BFA57FD0296BF98D0985FEC6D
:106560004861E9BA233F67B933A85C1D8A2E7C20B5
:10657000E734169E180B638521022479A02300407E
:106580008133DC942FFB993C5492B0BE5BC9D31C81
:1065900043B1DDD882327602251407C50DB09AA822
:1065A00040A8A51E3236A06AEE5A06EA45191373B2
:1065B00015D2793DCCA29E734506B0A8AC0C85607F
:1065C0005B162CD889E87C64A5CCFCDFF9AC69CEDD
:1065D0006D5B587537C847ABC306D05F490DF7D31D
:1065E000728C03EE6C76DFD400858D59558EDC03FA
:1065F000D6F46B0DECD3879CB706E117A13110ECF4
:10660000D4887F1F10CA9FC23E76045E1638315A66
:106610000F1949812919BDDE16F74461A154A2E57D
:10662000ED29ADA66BBA4C0BB86D36E573F5422576
:106630007B305B05AE43AA9562856B34907EA48166
:10664000B93B436644837252D0B598FB7C73D92022
:1066500076A23A827F51C2274FDC7FBB3A9ACD3F68
:10666000BD4DDBE778C921983DCD24CD2698FB0BA5
:106670004161E9A65592AE9DC6A681AAC9E86FCA36
:1066800034249BA239A3319056AC2FFE5593AB5EB8
:10669000AFDBAC7A01AF54C39C2A9848FCB72DB647
:1066A000599244519B31D9D9AD96415335D4C9083B
:1066B000BC6EFF4C04052A595B084DCBD85EE3F055
:1066C0004527E204E16D1CBEF4C273E99F818CF89A
:1066D00066229A6D0C32D98B088E4F8419611A2F5D
:1066E000C61CFC225919B13550CADEB8B48E39C562
:1066F0008652776910C45319A4391728409DE89C25
:1067000034CDE74EFDA3AB571ACDE49B6787A4D6E3
:10671000975534F9F710871B6628B1090B342D966D
:1067200097B2EE0A76879DEFC602940373943DD923
:10673000D2F69ABD50E96EA6D70ABAFCBC8E6E4559
:10674000B0AFC5DDD8214F448AEF678FD6D734C9A3
:1067500020A68C6DC459CD6C6D5171B1691A45A7D5
:106760009C15BB56A10CF2318E1A0411C7EED93D0F
:10677000CA1EEF4DE5F968A3B5D55CC5C16A188698
:1067800075FACDEC04F0466687DB66C2F97A8E02B4
:106790005516C4B08DC970E57C1E4D56F86CF1726B
:1067A00029CA4820B8C0DC4D72A4F7ACA54A4DED0B
:1067B00002DE7E4E9E8727BDC8F7A2658A4FE9ECB0
:1067C000E338336F6BB7B8AC9AA5FD068DE255B7C9
:1067D000BD0D51CADBF620490882928C113F46322A
:1067E000352BBC13E8B2B557CDD73C090B6F55A379
:1067F000BA423D2BE47A8C769718A79840096154E9
:10680000979F9313418D0E5A1D5793277273979933
:10681000AEC133EF4604FB402A8991186AF0D8C212
:1068200000D6DAD984DCCEACB8379BFFA463D0F2B3
:10683000EF862682331593FA87F931DD495CB55D21
:10684000AA46C9A7D3C5A3CAC2735E9E8018CD4C01
:106850002D6B9ED6C325B1365C49024F0FF6060557
:106860007FC5E755C164E8195A8C5C4C747F1008E9
:1068700042FDDF9C46F242BB3F5B993AF0E4EA19E5
:10688000FEB56A594ECF0D34D4424D88A93DF8F07B
:10689000BD47D88FCF48814A793F42D30B3E4CD376
:1068A000376D49F1DCD59909198CF57D6F5688B99A
:1068B0008AAC2246751DB5B6DD07FC115E295A0467
:1068C000A40861B492D62117D06B6871719BE3A4C0
:1068D000D0A5C4E5F091CEC357A5A372F926EABEB0
:1068E0006A72FF82447D6E09FC643D54AC8B607D0E
:1068F0005107216781A1FDEFEDF97896CA84E72B56
:10690000A8BD656900AEA6C08BF25EF5D21A1C5E0A
:106910006B2D87E1EB4331A0E997E40A55920BC652
:1069200033B8DEE4C2451C86EF3B9B8D38A25BF595
:10693000A2EDDE55A4EC8A18EBD67D26EB36404955
:10694000A1FAACC50DC5FC8B9D077F22F38D36AD3A
:10695000E521A2A4BA10D592DE0185218C23C0B016
:1069600040BB3F48814A2D7436E8A2762E508939C3
:1069700097C151434BB852B4A196006A8E8BE4780C
:1069800003D5E2DC39170B3E9084B824B2A9F11D7F
:106990003957D43715BD754290AD8BD8BE099505D2
:1069A000E7FAE5B1C667D7B191BC1ED46A671C246B
:1069B000219FAD6A689143F3E317B6E4B0630AF62A
:1069C000BE016F16FF8EB9BFB3723A54A98E35FD62
:1069D000033FBB9ECA6FA48BC3F343F5A07EA4DC28
:1069E000FD2761C11C0CE16A7F2CA21A3583B951C5
:1069F0007A9F471D14855E84E39F79513CE3633998
:106A00008D718F616AEA2251E7A255A199F1EA8955
:106A100086939C2B52DC0E89DCE2862C8749E4B8F5
:106A20008F223F907DE7EF369B12BE3D57610D25CB
:106A30005CD43CEE9E28859E6278FDD97E4C5942FE
:106A4000CD0A67A5BA2E7D304A389A0DCEDB1A30B2
:106A5000D6C9016F22A3F120CD1FF10C274659DBC7
:106A6000CAC16B9706164EC7C61E1E958EEC898747
:106A7000092D343A0056B5C6558F2B6456D5933D33
:106A80007586185530533627CCC5E4CD0582275975
:106A9000FF5FC0531407A7DF57CC327CDE66E203EA
:106AA000718EE0048E78A02F2BDCD8302427DE688E
:106AB00022FA86172E26902434CD9ABAF7BE64D7D0
:106AC000E68B3749A3E2905C798382609D4A1F0C74
:106AD000C099460263AE72E10F9472FB1BC17363EF
:106AE000F6E2D93096439D0E3D180A6727624CC9DD
:106AF0005BB0C26308C0AA8F51E44A4DEC6FF3CA81
:106B000022371E91ADA047E8BDE8EB903DB1B045FE
:106B10002B4F021C4FFD5C18A8B35EA7BE55D5B91C
:106B20008568EA58E8F308BF02B2CE6E9E96081355
:106B30002C30F207DD1346ABD83CB227B90CCCAFF2
:106B4000B1ADA929B8908304F4B68D4D200E15601F
:106B50007FDC8138D2E58A85AFC1A8EF2D0BAC92DE
:106B6000344346E9718546AF20B3EB0E3AC8332370
:106B700092D1C0F51F4EEE0C54B6FBDBD4FFF4C32C
:106B8000755A0629156CBBEE593A52F2DB370C7B6D
:106B9000B332FFE0EC03A857E58FB6CBBD93775037
:106BA0000DEA3EE7FDF697AF4E1394C31B5426E162
:106BB000914FCEEB43E9997C8E4AC28DD6C2EBCF82
:106BC000F311765AA26BF083EBAAC386858A744DC3
:106BD000AC32B1766C981BEECC1B5E7A31A29D81F3
:106BE00064A0FF211A43C92E56E2155BD51DF42679
:106BF000143E0CB18AE207A477861D0D061177E9D1
:106C0000CB18FC2FE4B58C0B6C676FEB26C2F766D4
:106C10002E4F8D820DEDF16C5A7E0A64123C590A9A
:106C200095BAB8DBB306F5099B3F3C67127B191395
:106C3000B6A9F7A5B694D07C96186B4674BA8BADFE
:106C400036AB2A98A2FB6F42B1F42D034AECB88709
:106C500027BF95B92BE53197A16990C25145CB2F3C
:106C60000FF4313BEB232E0C58CC507E1A13FAB2A2
:106C7000514E61D46A417B048FF176BE8F00681259
:106C80008C5FAECE046B19D1DE1068718B65A47277
:106C9000F36D5784586169DF2787A014E6EDEFCDC7
:106CA00094AF72A7FB6CD6E86220B90676DFA9DE46
:106CB0003071AFBA000E82560F9C9476484DAB9C53
:106CC000B87BF7A5A7758FCC73C5D4E393E02DBB34
:106CD000872A37D4A282768FFF915B5ACEBCF4BE4E
:106CE000A5B6107B52FB43B02E8F8EFDF8215A576C
:106CF0000C0B7F2BAF5227BD64283C5C0522DDECDA
:106D0000F09B7B5F60D0599FAE85962EACE302C7A7
:106D1000F331A3BE6524E3FC1EB4BD7D6DC326C65E
:106D2000F0FE240DEFDA60108B9FB70B989A9DA8A8
:106D30004FE131F45E1BBA37B4E15A8D94A77E61FE
:106D400067AD49D07124513B16F90575307620871F
:106D5000EEFAF4DC65C7315F197245027DA58779CB
:106D6000DADCFE3C5AB14080EA4132C816CC979931
:106D70002545BFB22F70B3A4683E5BB591B13DAD60
:106D8000E7182B34B446AE5CB6ABC5997195BA5CC6
:106D90005762198081E27CCEBD8C12622B2AC00A18
:106DA00040A61AEE79F06BF69B2F393E17E6438921
:106DB0004B6233B4DFB0DD983DB0A0F60C50223802
:106DC000708E9FA7251AEE4543E7C36F56BF15483F
:106DD000704B6D9E0591C82269D6183978095EB747
:106DE000F6AB9C80DDC82E324C039CFB1AD92DB526
:106DF0004F669C1D74A2DF9AEE27D8E66BFC802AB2
:106E000041F27F73B1953138A0CCD322E7C416216B
:106E1000508976133010BCFA861B2990FBF0EB47A3
:106E200084A67DE096BDF77137C91B9F45F13124DB
:106E300010B105083474342535D17CAE6695698A65
:106E4000315CEC6981F799E57F93CB24B687B9690A
:106E500080A6987FB8676C8E7CDC9B395C92198821
:106E6000ABB8EE3621B19240CAFC813958F0F965D1
:106E70004EDBBCCED225B7B47DC0315051B1C8B5C0
:106E8000BFE321C02E8304176068A78D363618151E
:106E90002BC28BB79E3B619FBB8B7506281C66354A
:106EA000C6A37D66B00E3A228B7D57446CDA241A55
:106EB0000E569D148F6B18D303FD168601A0905DAE
:106EC000D043329A7E0833A506265689D49DE5C85C
:106ED0002F3732F932A80584D659BC790FFD7BFBD8
:106EE000DFBA8F823163E4BCC4CA4F17719B5A0763
:106EF0005256E00AD00EE94D748E45434591341048
:106F0000EC348619B58563FFB8755CD67577ADDC52
:106F1000A60C07210767DE6EBEC49368B32756062A
:106F2000351822CBE4686E4A597BECD0A2D30135E8
:106F300091C72FA309D47B26D5A9898DE5FD5AA930
:106F400048CAD40D23A016A9F90AB56B49F6589F73
:106F5000CFDA88C44616C0DFF24B159B84BB90196C
:106F60008322CA497D6C5030E3A9CCEE2BE772082E
:106F70006F2994860C1106351281A54813CE270C73
:106F80002281370B884F4489702E69A8D116703B37
:106F90002D76A8F9D44FBB9E841558F89D363B6ECC
:106FA00068C9627DC38A75129411A65A77A3776B5C
:106FB0006C660CF175113F197A6A262B627C4E368D
:106FC00065453E4362C8CDF77D5A5D7A7326D97B0D
:106FD000E4ACA4FD84B75499EA25D2683982359F80
:106FE00013201E93D05DAB11D69AFDAC0B69F4ACA7
:106FF0001E5D7E0D82E59D77BED085CC936EDFD77A
:10700000BE8B367C9F04739EE9875B58A8D8822884
:1070100061D9C1057612129261F785F5FA1911D579
:107020003165DB48F9C4A5C8FE76EFE17461220A38
:1070300035ABC5E6B13DE74EBB1BC0D330247C3E2B
:107040005049ECA51D4387BB97DEB34FD8415ADDAD
:10705000D366D571BB9D062D750BB76C3C0FE760F1
:1070600003BF3BBEBD3C1782EE4CE24AD9FB66FE35
:1070700048862CC9F8BFF84440F867D795517B7A09
:10708000970596C1F7E9C1F5B9F3D6F78A9EBB9784
:10709000E8B0A611EAD6FDCEC7A9B6960A1E97A9F2
:1070A000FF5B78D5056BAB5F5C945C0A1A2CBA87E2
:1070B000AD471240B0B71327FFBB0DFCFE4D60700B
:1070C0001C0248241364BA0AE18F003010E32F57E2
:1070D000038D7E9B79A3055C1AE8B600C5EF06E038
:1070E000A073E444BBB5EE5E1C58954B033EDD42F5
:1070F00098756796EB2B13C8303B5916CDC9F260D3
:10710000E85E8D0D7C84798804EE306EC923B8C4A6
:1071100093D8B4B1AF09611C20CB7FB5B8685E3D90
:10712000C0EC772042C4D6C5BC8B5F7114405B6A4B
:10713000B9B3D75B6BC0D021CDD8A55F446EB28EFA
:107140008AEC76F38B0EDE8B68A8EB608B0B65E721
:10715000711EE0B69BCCC274685ED81F628CC85F9B
:10716000FD776FD855DC56FD1F6FBB153AF11DA397
:10717000F0575318C681E10AB9929EF528D1C7FE8F
:10718000E37A155AB14E259723D1C4C07A542ECD37
:10719000123C0C58BA78D715420BA4BFD046B60A99
:1071A00071992EA1F71EFB011ED27D00069A1F3594
:1071B0005A0DAF6BC9CC2332BF95099E77E799A5CD
:1071C00015FE56041D81FFEDE66E3171944AEEBC4A
:1071D000C0E6DEDC5405C33A4EC2A88481DC70658B
:1071E000779D063CAC7BE08390CB19B30B626CC5FA
:1071F0001DDFB814C1C80C25466601479A39CB4536
:1072000025D15AC9CEB73AE86EDC0AE57B30774320
:10721000F71606F8D3E64F4CBCE02E4681B3D7C52F
:1072200018E7CF36C26F85AE788A6854B77F8B3E39
:107230004FC96A7477586F0B6F7E02D050D9871789
:1072400084C163ED039DB8804512FF762551A44E9D
:10725000D1F32939AE1D9BD960039FDCD096082954
:10726000E08ECB494AF1EEE94323E7322DEBB56CD2
:10727000243771F7885662E83FAC5AFF096288717B
:107280003F4E7D189F841147A58679EDA9E05DE208
:107290004A00BFC854E382C2C8D159978143A9C9E3
:1072A000674AE467091ECEE9B8D417EE2B36A980E9
:1072B00038A5A469B5D6B2DC0C3667A8A6FC36871B
:1072C000513E8ACE82386C1C4129EE5D047B0A0255
:1072D0000D035AC109C300AF6651921D9858C313DC
:1072E000CA20EEDCA82A9067B746B74649854A7B94
:1072F0003EFB601DC88D577CBB881610AA441576CE
:10730000FAC00653A245A3B167CE6EBF36D65E461D
:10731000CD3EBA3AA92486513D0EF7F9F74767F0FA
:10732000ABE5214D21509942AE88A5B365F9706156
:107330008902562222F63BDEAA7B9279B0C85E2FE4
:10734000500B9D792E0ED8B5307D81FF0267342D0C
:10735000E43EBBCFE344F3FF1BC3339649C4374637
:10736000976D687D35B11DDA753165CEF313ACBF0D
:10737000F0459BAC29ADA093065B53819F0FC47B66
:107380004DED842E810B101B4869C5051BAC6908A7
:1073900090E9F8C0FBA81AF76B623CB508E11379D5
:1073A000D055C1FC521FC81C860C7A763225563047
:1073B000629C43A33641AE9B8E5F5313970DFC5FD7
:1073C000BB3E7953815D3E5DE8B3B2F1771E14B3E5
:1073D0005F2E659A29268A7960FFF38E6E1408461F
:1073E0005354A58847B6ADE801A8ADACE803B2AFE9
:1073F000431157AA4848CC90CED0D6D0FEDA976039
:10740000D72BDDDE85E9348386622D717512781EF7
:1074100021406F8C35ABA838EE6F78CF9A313E2F74
:107420003D6327EBE3F829D1675C52CEC52F9A1B49
:10743000B60849A94FB37F7CD4EDE72D7A31C0C49B
:10744000D1BB86C9A6752947F5C55CF6923DCCB57A
:107450004320F32C29C83111B128E6AD59A5380FC6
:10746000640D12F1DFFC9F0292855760B86291A60D
:10747000D0838997A1BD1A6BA52890BC86596BAAA9
:107480001EE72B42DDB32F28B5A6AE626DACC987CF
:10749000C9323E3CB3727C6960EB684DFBD2191572
:1074A000DFD965557FAFBA0E5D073D05C8433D7511
:1074B000DF1FA2139D99BB853D6C73EF59969F67A3
:1074C0007E7860F9CA8FE5016EC25F49A124A77575
:1074D000E1F6B184F6BA49AF822C4901A235C8CA97
:1074E000E7CCA10C5B9BE0FA8576A1AB6599B86609
:1074F0004AF14FEA5C01B476D8462732779E19AE3E
:107500004DFE616FDA939A664BC9CF78AC79F888F3
:1075100029D4FF40890B7296AAEAB4192130FBCA1C
:10752000796C8A89C7EFA8D827DE82CB2EF96359F8
:107530009665CFC1D86E724ACC31B8D5498B958F3C
:10754000A09B6383E3631964233D224C963A355430
:107550003FC0E3490F08BC69A10D48B58B0831FD58
:107560002C2AE65896D88E816DE61CAA75EED5E3D6
:107570001C04B416EC027C607945C321D060A3FFE3
:10758000576BCD5EA0B13DC228AF46995D6D43D12A
:1075900024946607BA67D24FCEA599174219AFD780
:1075A00017222D6BE6D58605DC2966E554BED96326
:1075B000E10847BCCF8B18A9A14FE0E3981D6239C1
:1075C0000AAF22E802298D181C5A8BA48AF6EE17FE
:1075D000A966E1AEAC7EA6AA6A723CC9F76950BE44
:1075E000F9FA197E63D0D9FEB0F351BC7ED9F1E32C
:1075F000A8A0E862CD10647377548714FBB4594B8C
:10760000D72813742C7B31C85E0978A56025770DC7
:10761000A2F0DED492D796B963989C76C390374592
:107620007592E530702704A69C8B77FD0902D795EB
:1076300057F07AA80157B657E5422F810100A130D3
:10764000F1C8B70D4E5866C23D6DDEB1F4AC068090
:10765000234B1FDEA8A066B97D87184D8AF5608D83
:1076600029A43941076D81399A1F5D780A0FEF15FA
:10767000EA843C7753FF1D0D755737F25C53B08693
:107680004F7F3D24AB2F4ED6961011383579F659E1
:1076900047A1C0C58B81B09945F3792E85AA5FE7D4
:1076A000D7389A3393E199E92CA908B602117B28BF
:1076B000861649CBE98A9F5266C27E6FA997AEB102
:1076C000ADDA70F3BEE2573B8F73FDFA81796951F1
:1076D00047CEAE782BB25FFF518B24536EA9274360
:1076E0005C1376470784B9B02F1BCEA5885E4D1674
:1076F000156A753F6EA947D1074DAA7563C4123844
:10770000C71F5F00E7F5D2A8928A76D85699469CA3
:107710006D5E49405BAB672AD61DDFB3D47806A106
:10772000CFDA654840315930A07C600B2B187CC4FF
:1077300015DCC5837841B6A4BA26BE871AD986E07F
:10774000D43D3E98684FECCB3B2D1366358024EE3C
:1077500098362FC0BC568DC2DDC6CC96B0CD704BCE
:10776000E6A75D86B04D171C69132CBE8786AAE07C
:1077700082629336DD98F7FDEE496CC9818F5EA376
:107780003A5449F2655DCB8629A1CC1CB47799ACFB
:1077900099D4431311B2911A4B092F91C007C96BA9
:1077A000D4C92E060C522DAF9A9A6D12AF00C65452
:1077B000B59DB74331FCC35EEF93BB8E46F2272ADB
:1077C000D37C111365B345C99282E092FC4009A6AF
:1077D000C7B2495A962D6AF1C401619C771B92EB9E
:1077E0008440391A4EF063C41B6C6DE056BBE31540
:1077F000C3B8C3293478CFD5F64E0AA50131387104
:1078000091C253AF5DEAE3DBC60D84815ECCF4B672
:10781000129CE0C8EE8758269AC1252B214D9A72FA
:10782000D14ABF0C1877E358ECFA6FFDB71D32A3AD
:107830004F4128118144038075E538B1D939FDB72E
:10784000C72FEFF2187D4EEEC48BEC8D5BAE1FF2AE
:107850003EBA4902A14DE1B4B16A79C329B1F1E25E
:107860004FDC8059A0148AE349713CE52B774EC464
:10787000F844FE4975BD3EBF6D6DEBF8EDAB6BC0D6
:107880009524FCB7EA65C607E58F177490163C533C
:1078900093BD9B0A4F122CBDC415B1D307B3074249
:1078A000D8F4FF9933A5AC851126263CA9442F16A0
:1078B000A37F778603BD60F002EA89424F7DA4A1D1
:1078C0003A5CABCDC110FE37BEC58C90C31F32B33E
:1078D0000CFA3FBFFE6241BBE514F1793A38E86823
:1078E00095D5A65E63CA449D6CAE7D742E163FA8E6
:1078F000BA03076FA256BDD317B4A7DFDBCD6487E9
:107900003DC73FFA358759ED9D04A7B00FB3B9497C
:107910005B692DF031D1C80E36BFB606BC0289298D
:10792000B47DFD1F4B81D08E1335C8AB66B2E02706
:10793000A6E4656939A211122777A50FB4706865AE
:107940008F28F08EA9C965E59432335DB834168D61
:10795000CE438F6070C410F6DBEF8EBE15D4C89393
:10796000A6DA077FE5C1A7BA2F736F636C6721168C
:107970002389AE294291942577CB78B9FFEBD61BAA
:10798000A8D2FAB5B157C065E58433F2A4110BA7AC
:10799000F33569C7AE7FE7144EB40A7D2BFB84A88C
:1079A0009010A664887AB717A0D74CE2940EC6EA66
:1079B00046D9B8D780F1340806837512FCB6AA5BA5
:1079C0007F367DF7A2F8D0311E0654E0F212577BC5
:1079D000FD9D796FFFA3390DCFCA99D4FFD260C244
:1079E000C62D65778271879902890E895FBFED1375
:1079F000D54EF80AC0C97F5E3A522DB38648907FB3
:107A000004E2A694779FF42BBD1A4F966A86BC3881
:107A10003376EF9BF8660B94A3BFCFC651273DB3D7
:107A200007C787D760876BECB19D8BAC0E6FDF48C3
:107A30001EC6A43C0681283C165EC6659D66E3A76B
:107A4000B0CD58F112FE55354DF4A6A6E8691D4596
:107A50004D72AB682AA79A7C468A6DF906D296E6E3
:107A6000A7A7672BDFB9F6C17083A3C7AED3A75111
:107A700004A834E0662AB00155F6CBAA2A374BFB9E
:107A8000B40403742FD7456105A917369CC58A7ABB
:107A9000AEEE22C4422F1A8D5B3DA7E2DC75FDF5E8
:107AA0000DBE053439EABC634EC85DDCBC0F9CDA00
:107AB000318497825BE03B1A6776FC886DB7FEF2F3
:107AC0003F214F5A5BD7BCAE740C4D562BCFA56BE4
:107AD000E90543A838EAA0872C34718238CE046BBC
:107AE000DB26DEDC161FF28B51693EDA444670C19C
:107AF0003BB4BA7E36AE1A98FB1657D3C2EDDE40C1
:107B0000FDAA541FFE0000013A8B56B79299646B90
:107B100028D458EE165800812E2AB3BD948571885A
:107B2000077E03A0026F51E549AC34D6448193E54A
:107B30000995C9E3D008E82BA0E663021BD739B446
:107B4000227842AD2C41C5EBA21C3715015B048A9B
:107B500097E788871DC78FF921D30BAC24B0446BFE
:107B6000310F054E40A90DD9124035570B4C0B4D26
:107B70001619672830C5775E42EF75C810A76AD717
:107B80009E6EDC2FD95BAA106AB2F706AAF235E224
:107B9000053CE67624AEB102A87449E59D8D200A25
:107BA000D09FB072CF84CCDAF869245C170A7F2AA0
:107BB0002FAF2D712DF99381E8ABCC6BEB45C93A12
:107BC00090F7CFF35A6A084FCDA7CC0050BC0649B6
:107BD0006263D372CB76E426D308959C94D824B004
:107BE00082913F3C179300F8DA3929C0843D708FA9
:107BF000C3D12B4FD4BA1FF477E7E8D148FEF498ED
:107C000028A68A6AC27E933D308A0E413341277589
:107C10000E8DBB2709049E1B25A77CA9EB65491B7C
:107C2000D35B267090612B9CCCBA820AFF1BB65B9B
:107C300089FAB8EB2457B25D80CAB786E619639516
:107C4000D4868773FDA0B5DDCCF3389E161EC6F032
:107C5000800BFBEF0163FF70FB86BD946BD8C550B2
:107C600024302AAE7D30162945C19D7D1C4BF9C7B5
:107C700084B8C5B972CF0CC20B94D9160BD131C0E0
:107C8000C18020CCE7A69D94748EC626B7623C6B5B
:107C9000525BF772145DAE67A6B2248AFAA12DD8A2
:107CA000508CB8931DBFEF7373DD44E8F4CB7F7045
:107CB00066C6D6E6ECD30A4C26DF212DBBF2DE6881
:107CC0009E8EBCCC6F30983B2A0F4CAD8109F55D80
:107CD0008833323357828618445ECBB1FFE54C03BC
:107CE000CF8BC433D3502ED8568436B4FE7A8476E4
:107CF000B57C0DCB0F45870E9FF2158AF5C7FF03A4
:107D0000F143DD2C417157A06139B507E479834B0C
:107D10002E370339BD17B0F9982D51635DD5D1B118
:107D20001FED015244C5E3142F156C368622D3D1C2
:107D30003BDEE795F9C78F1F30264B4818BF10A2CE
:107D4000EF0E5726E9127C5DFE95B7881A5F5BAA95
:107D50006DA5C801B68F2C30D8655F487D3AF3DC3D
:107D60004C2AE91BF22E7F62A7DBAF984CC412D5D8
:107D7000157DDFADE867BF676635B938DD33AA54D6
:107D80006C73F026A763B3BFD2E8B388B643F9CECD
:107D90006231C3E580EB9E77C71285CEDA5E9B5CCD
:107DA0007157565E07DEBDA7DA9B959B5E7C68AC7B
:107DB000FD9AAD123AD4818B6834465F9236AF4C4F
:107DC0000EF35508B5F0FAF47BB87709543CE8EAAD
:107DD0002A62476F8D3DC26A3D4FD11E951B0F84AD
:107DE000EAA6831140AE3A11B9FDB49F759566EBD2
:107DF00004EC22389BDFC4FBE15F1D793B3CAE19EC
:107E0000F4517AE39323293057AAE937E9D7EB9B5A
:107E1000DC45E92DF47786FF1DD71B3B67BEC7FD08
:107E200051928E46E98064E6B062ED0347B63D1993
:107E3000D95DBC629C0819443BFB558AF838431A4B
:107E4000374FA1646D2A41FAC11D478A5019FC348D
:107E50008F4869AE1F55EE24BC1C75FE703FF318A9
:107E6000378FE5BC6A7AD436FDEE04987565C9177C
:107E7000B1FB1E8651FF8960F73B69B0D0F5B02891
:107E80009F60B811447B5742A39CBA515EAE2EC48A
:107E9000D35FAB5BED4908DC0CBECF4F9CD436B250
:107EA0007AA2660A6DF3A28D7B5E28C9B49C962CDB
:107EB00088D9D95B2F48561DDC1CD4C3C2E6631E8B
:107EC00093D330A9121AC6D1BF84EB2B2CC1F98EE3
:107ED000ACC3401BF5736685848D690D4A556BD81C
:107EE0000BA1D1A49E6A5D2F0DFA765DE65392290F
:107EF000751B59F92E99DDB659C23ACF4126A2A376
:107F0000891A8548957B6EBFF3CE25513B3F3DB323
:107F1000E0A5D3C0A84647B8F3FCD04CCA6F773B66
:107F2000DA4D7BFBD4FE1904B2AF3660018548B050
:107F300012BCAD8D56E2DF095D839CB859AF0CAD24
:107F4000BE89FF1C7B3B7E4C7BEB0CB7EA0289EEC3
:107F50006C040206EAD87C70FDB6B35AC66AC52323
:107F600009F9F86DF23A6CF24E2A9EC1AB517C3F92
:107F700062655D7E8F5071E0F70C5AEA93AA98868D
:107F800010D084F6C588F2D04F4F5A529A0FE1E0D4
:107F9000A74ABC173665981D0B03EE2301CFFC31B1
:107FA000BDF24E0D3A82C6FF67207BF8967E89A10E
:107FB00027BEDE934BEC5067D66AFDF3C47A1002FD
:107FC000E485DBDA2CB9FFED16D9EAA7CF9DBB70AB
:107FD0000234E13A73198022F3B166C3E09D98360A
:107FE0009DB668C52A4ABACC24E467A1868C9C3C1D
:107FF000D6FDE6C1CB7CFF0AB9552E8E31D5067E63
:108000001199E34A512DEC603938DB493FBBD43F2D
:10801000E400DA3E74B807F95C7E111BD33427768E
:10802000A415DCA1B2DF69FA6B992251462EF3B296
:1080300045747AAC408FB663BB1B720CD91E8CFEA4
:10804000F60B79EEBD602764F1C86A1F70467C822A
:108050000D36B68C9E71D566F39BBE43D98FE4BBBB
:10806000D602F9B557CC449C6A640E5483837D0FC5
:1080700089801F795B46B23F11F5E992DC10A5ECCF
:1080800096DC0210C5FE853AC184699D8E8E7959B1
:108090006912D93B15A89B40DDC7DD358BE2A1579E
:1080A000343D8E768CFB7A6A95E2E4C19316408863
:1080B000828EA6B5B89EEBD2E39B1C0B9F53B29E5B
:1080C000D3DC7EB1650BE6261A32816EA8CE2B3C3E
:1080D000947477A4C8E1866D56CC985648EE33A1C7
:1080E000C76B1F16E0D133D891906E22FB5BBB9615
:1080F0000D6E29A8C08806BB9207F53DD533B77A27
:1081000093F774C6911E5CB14896304643955B4B1D
:108110007204EA9AE85549EDE01656AC41CDF69C5A
:10812000CC037C0A5947F49F11ED3990016F342834
:108130005729CC8B84F57983C6D8B6F6835B740255
:10814000659B010BFC6BD38FAAF81787EAF5437088
:10815000C723E68CEFD0D03F0D8A12AB6108D85D03
:10816000DC04616DFC0C927063690D04E160C7C9A9
:1081700066DA76405FD0B76AC9720F2839FFE76BBD
:1081800032A99384FA758FE3B688A3DC026522DFF7
:108190009CD2CC727EE8831677C8809BE214B97FAC
:1081A0001CD9AC7F152CF185F05CB403B989A52CE2
:1081B000393A59530B15C67426370E9A17A3DBB5F7
:1081C000AB0742962A16A8D731C72760183C3770EC
:1081D0000B8CF79FF6CBF35E8F70F74E8F815CBBF5
:1081E000973FCB174A1DC133EBE19B7AED4E1569E2
:1081F0001FB6B1943148CC8EAB295112946B03CB8E
:108200001AFD61F546365D301080666DBC0157D3AE
:10821000B4F793E5127BBAEDA913F1A40C3EDCBDD3
:1082200009EB025618A68046404DDD7B8B482C8218
:10823000588B7D683588F9F50944D97127EDDEF151
:10824000CA2E4D2AD706EC9461AAD967061D1212D0
:10825000FC8EA5E42AAEB1E021CD950FCF214FF4DD
:10826000F98277F32466C1156D207111FC2BE12989
:10827000CE02389343A301406E6174317869F806E9
:108280006390A774B114E2149B9DDC9ABC3F916A81
:108290004C560E66B0EEAE991F7BC132275AEF01E5
:1082A000A96F4636B9BB47D27396430B82722CC175
:1082B000D83DAF809743A08CB5EDAA3643DD86F854
:1082C000C39A0B66911F86E090A52E2D18198C2756
:1082D0000FE6E24F0755F94E238FFEF22ADA110A14
:1082E000D86680C9B75875973B0E112EB215A3B04A
:1082F0000E2CF00400A2B2405BC09539F6051C8339
:108300006640DC51121A0EDC0DE7245E865E3822D0
:1083100080444951DB76BA4B3024141B7A78000F25
:108320007CF97F1EB9942ADEDC7DDA4829566F5924
:108330007A82274B811775A5D0C1CDA786DCE9814C
:108340001B644F4D0A4C21A35042EEBAEE48914DAA
:1083500044F0A8117F79D9ECA5374E02BA8A208E55
:10836000E81BDE72AEB5E42B8ABA439523738914F9
:10837000F32BB78158764038375A4E5F274530A1E6
:108380002A8EFF40C5B603A7A98DAAD19C955CABE8
:1083900089DA527C5327D7646843479D611280FF76
:1083A000E0A8E38CD62863DFBCE8A2EDBEA2439F21
:1083B0001AE0945D4BDC1A11AECF2EBDBA8CBE0212
:1083C0003EC2BC1F0E3033E8398F3D6CE6B9A719A9
:1083D0004DC3A6EF985D65554330784DA0A0E626C5
:1083E000F1B87A04C1FD65A57E2D2566AA1658DA76
:1083F000E5E8E8E3063FA3BB7DA41C44185CE70660
:108400000E9A62EC507B6F087C3FC9FA7B0EF5A494
:10841000BB6563C1BBEE2DAEBEF9188EADA293C590
:10842000FD9E7415169FA2742B03046B69DFC87D33
:108430005FADB13EEDB4EA5E6C0C15903A03705638
:10844000623A475416424A8A2FAD98BF52FA013019
:10845000952B8295C7F2AF77AB12AB3BF4FD5591EC
:1084600081FC272A8FF40174B0B1ABD041D0F172F6
:1084700089B4E78D2B52B76DA74899345CE5512A32
:108480004BD450C77481658160D8F5806AC45C03A1
:10849000D9FDBED6B2F3CA4708A757010494869CFB
:1084A00076C388D37A4E08CB6672B8C7B43D4E30D7
:1084B00062E4DE2FFFCEF5412E0BCFD8B64908CFB0
:1084C0006492B3D2F5620AAE87A19E0E921E45E376
:1084D0006B399DCA6F35BF30BCA62A10ED87288343
:1084E000348EB8C8D4491B5DD92D4E36E6A8EA5261
:1084F000E8043884EE9AAD1AD49CBBF40AA00ED5D9
:108500006C2F0ED8AF47E1F903FD3C1F67782F5B56
:10851000A85276345A73A7276EAB48BD34FDE6EDFA
:10852000545CAF0532800873B24D71DCD9267C8A69
:10853000058A6EAFB7FF06ED0C2CB8AE1E92E5CAE9
:108540005F65941E7FFBFFF9032F993C243AC74CCB
:10855000DBB9BF0DA36040F9FDB120BE3D295BC270
:10856000362837A859376098C0E848F86807B6B089
:108570007552D83A7F8744243A64A0CE7E52A9DC53
:10858000F5862A22F8FB3E95CE12F6338A57C4852B
:10859000720A6A51FF73E1955D6C25745999F16B0C
:1085A000F00578533ED39B9E172F8098797CDDA2EF
:1085B000006137557E0A5822BDE0242C18AC446572
:1085C000DB9E7CAD4574A95D830C3953F9A84462E8
:1085D00058486568AD97A0BAE47003EC636CE8D7BF
:1085E000CF0F0396956408A4923FEC2D4A908E70AD
:1085F00063E02ACCC61C4A5623412CC8C0DC9B77BA
:108600002037C6A8291B358C866A4F4CEF05F3B975
:108610002103F4DB6BF5B958BC91E62EAE26A843D6
:1086200067EC0D65B6903E50AFFD8AD99496C07741
:10863000E7F847A3E8FC3620B9BCE9E8E7021F9851
:10864000AB56623D58FDB1B6C8763B42CE3555E7D4
:10865000F0116EF846713187825C25365D5BFA93C6
:108660009A8AAA26AAA0622201131CA4C845B2AD08
:108670007EE1DB44F1B64A55C395FABEF1B60F6808
:108680006541604FA5D4DA91FE8BCF043CEBC44D1D
:10869000AA1BA89F7053D0C3D02342C911F1E64949
:1086A000D2BB15D935D8FE2946E4ECB7D84D6504C0
:1086B000686563E35AB0F4E9435C5BD517E0B3BE89
:1086C000D1BAE5742D669BC787BF4BEEE31E3AF522
:1086D000F864D82195AFD537A7385B012BDCD99842
:1086E0005F29AA8C376C0AD73F6FF2430B2CCBFC67
:1086F000BB34DAE1C7CFAC45176836ED44EFDDF4A3
:10870000A9E68645E2200A3E6C3BBA7195BE3FD38E
:10871000BED4F3C4B624D966C2555A9CCEBBD47419
:108720000EB1A5ACA9ACE506701033C30541E8FD58
:10873000703AC0FA7F6F6036E9D1F41860F4C198DE
:10874000FD81CCFC2AB14C15FA5219C904B648AACD
:10875000988CE17915882235CA2F4DD19605FBA852
:10876000EBA461D6803ED1A73D44ED49B0AB1F5983
:108770009915B6D75626AEDFBE049A19ACBDCE25E4
:108780001FDBB65AF2B9102E00DB10979BFE75CA9C
:108790005839D6DC6894A2F3C38273591E5A18A4C0
:1087A0009ACBB5B9FC6B19A134C619AABD400A6CA5
:1087B00013D39BB66BD5E7D471797D501669062B20
:1087C000E12984286585A6DF9510D3F9CC3429DD0D
:1087D0003854A62D6A4036CB4ECFA7741BED5DC42E
:1087E0006541FF8AEDC3FCBF4D66C459BAE5E5AFEC
:1087F000494E9ECB44616D67ADD991A4B1A3910A56
:10880000A86E431DB9613F1BFB5786D116AD8A8503
:108810000686F83B2DB39742E975E93FC4EAD17B60
:1088200076B770506EDAE9B4EAC4DC8ADCD3AA7F8A
:10883000CDBC538712CD28F7D3A89C9C5119D3A047
:108840001A0D2AA3EEC7F75FD2AAD71C38BAAF24F5
:10885000511B0842E3C970195D25EC70A49EEB1E04
:108860007A412B477AA2AE75E6685ECAE86D3EB9DA
:1088700011A4999BC49A2671C9F8903ECAD4B23FFC
:108880002E2667827252B662D8AF9115B01A006A6E
:10889000AE5C229A81BD2D98495445D5B6C7E8EE05
:1088A0008A4E243215ED6E7836096109052047D8C5
:1088B000879E1F2697389D8F3A9D7494A23D79C458
:1088C000D2550F2C14563515F3D804CDFEC6914C55
:1088D00026A4139E1FE1D39C1DFE392FDE2B0A71A7
:1088E0004527AD989BF0AD38CF63B9969ADF98993C
:1088F0007DCB7E5FA459026181248A6329C3CDF3B5
:10890000E7CFFE696DBD4BEE4DA134AE6A36D0287F
:108910003904F9E51BF65D9066450D170A360A59CC
:1089200032A1955C171F385997A61E02829ADAC6A3
:10893000F0CE73267085DA588A247E7DD34A7EF283
:108940000DECD9762405A53F84AE39416A0FE9A71D
:1089500096D4C9299AEABE654032A92711243E8CD3
:1089600025758544E03D77DF8547AFA83EA0EA1E28
:108970003CC328F19352988B9138DDC44359C315F9
:10898000513CA9C34420A9336BB1DBF15499F701E1
:10899000E2C9D4224E89D1DC5DCA5ED2843AB4B831
:1089A000DD7B3BFE94F32A35269A390ED72A03063F
:1089B000659314809D0C53D8DD24F7B7CDAE6321A9
:1089C00050DD8C1FD2FFF28F32F24637314C105BF4
:1089D000F980F5A7B3539EAD5AAC68F3BF64251A6E
:1089E00053A00376697ACA53ACD263FB7B21F4CEE1
:1089F0005DE886A57C9E78ACF90BAD05BD9745DAA0
:108A0000999361F5091927CE39F9F4ABA9E1351D20
:108A1000864833B298A1EB227843AB165D269115B8
:108A20000DD5B9709187C0AA58D86BC55819601A6E
:108A30000CAB07B937FD0EC5E185F7D4581BBB7BDE
:108A40004E855170211F902C7192D965A16610B985
:108A500072D0A1B79D4B2EA076242D5A13F35F4CF4
:108A60000126DFC80DABD2D4F844611DD363A9E45D
:108A7000AF0B47B29FFC7683771FFE6D141661AB78
:108A8000CBDDBFA1C6E376DAF5CA556BBA3D427BB2
:108A90001261558CB1B74D0B798EE7555CB7D50F88
:108AA00052E6B2B51FB4F3AE768317970FD1F1BE7D
:108AB000F81B5A3747F31C745059BD95A06671E6F0
:108AC000C75599BE71E3579116E789E6FF91E751C3
:108AD000EDEA2EC47377BB30C6EC66AC1EB91E57E8
:108AE000FD20FA29E4457B9F0912198C66E5C19F98
:108AF000C1CA657104ABA2E17B31644C370C14AF81
:108B000060739042A99934DEA89117C585D09F164D
:108B1000242FE19A21E6C569A2228F486B7637059A
:108B2000C949D1A3A1B9B1D0F0A9DF95D038B29786
:108B3000602E7ED1515D653E115853D3E9A9D56BA6
:108B4000EC155FBC34BE16F3D3980669C026960EAA
:108B50007D9DC0E7BD73D1664A3BFB6F2A90C5C4BB
:108B600088BF0791C546B0AE1269CCE02498CEE329
:108B7000FB6EA08127CF3A936D759AE5038C92F630
:108B8000370F878B8995AE76C1431634B3A597848A
:108B9000F027603D11593AD116CD7A3D78F94087DA
:108BA0009EA15EB8B651852685EDC37CD99EF56041
:108BB00040DF9EEF8ECA5161EA5A2E765EDC427724
:108BC00015A044E444546A065C7B2400F8E1E2C941
:108BD000C38D0073F7F4E761D265E3482E28402681
:108BE000F2D17C41540F0A0CD895B4FBABFC39FB95
:108BF000F0D810AA9377EC389EC73D4191A2C0A24D
:108C00007BF902A5FC487706D62221AF9362AAB968
:108C1000BF3122BDB958632ABFBDE4AA6B8E7594DB
:108C200010BB5907222762A1497C9485769FB09C8E
:108C300030F7F7D3F50FDA26B57EB197DC09461188
:108C4000736FB7CD90AFE1A8128682A39931CF4B55
:108C5000A07718B5D5F0CED825CCB7CE4F6F2DCF95
:108C6000626A64716269870BDAEE6E070683AB1D78
:108C7000AE67E9530C342286E98A14EE2355204B63
:108C8000B9EC79A8130947F9150E78EBE4765D3352
:108C9000A240C5EDA22A0E90AC6247610F0ED97AB0
:108CA000EE21EEDF6671F6515659119D73707454C2
:108CB000A4FE57707A31C860FAEB4BD9D31414C5AF
:108CC000DFA0514CEFB0A520DFD8F0006863D84397
:108CD000EA0214D134F295FC911B76CD341453B5CD
:108CE0005923F624B245B5DA21B9E287A68DFD8C69
:108CF0003FF8BCA038886B1386B923ADB27FB25859
:108D00006D6A7E75E154E1E63F240B435CD4CCD41C
:108D100031CE6FE064F74B12EE12D011F16F454384
:108D2000152DD3188314DF95809916649D1164EE78
:108D3000AB10FC1450BB4E89CFAAE5077E5717C570
:108D4000C5CFBEC08AC1D5E446295FCC4DB1AF6363
:108D5000DB488CFAA68C4BE30116109E9B122FD495
:108D600071894EB1B2FFB2C103AD9E03F7830A49C8
:108D7000C7E49A7EC258EC91415F4250DBCB40E899
:108D80001B808B760BEBB17E3DFBE4080EE422FDED
:108D900037BF6AB1419D71BC14C419CEAE42FE27E3
:108DA000AA21B9EED3973B7291D3E352E746C44A66
:108DB00073AEDCD6689927A992AD59828DE8981ECA
:108DC0009B9345B5B61420BA833D5F28FC02086E1C
:108DD000DBB219B87368ABB5FC5D4103C5005CC478
:108DE000B6A3E67F32854E5DE6AE655A96B7C443BC
:108DF00001A52C0AA80587BCDC0387176C732757CD
:108E000038F2649AB64AF1C906AD8EE9E0178E22AF
:108E1000C7A78B698C6C9989D8674D35B2852FEAC5
:108E20004CABE73EE48351DA5283CEE2AE205B7076
:108E3000E6A8FD08F18B1E39666B738E75C1A5B867
:108E400005A3C812C8CFD47231C09A122FB0FEF158
:108E50008B05CC00E918B98735D15E060B57D218BF
:108E60002C1A30E5FB83D644A8ACFDAF91AE8F8EB3
:108E7000FA1A161B768FA340B22F981ECA8B8857FA
:108E8000C7AB8CB8587148C895880BDAF62CC2630A
:108E9000E333769D9DF00F20647415BEEEDF6017FE
:108EA0001F6AA35AF7AECC60DDA4835F68BA183896
:108EB000AC27BA96BC28785A99FF89BF35297249E0
:108EC0008D9CC4FC41874C4E66C0F21DEBFCDD95C9
:108ED00002253A0E5B4A1FFAF4C29CE31D3EAABA71
:108EE000E6FC3907838B9F12B9CA52E16549546C7D
:108EF00077669686FECF22A0A57ABAAD22402D0FC6
:108F00009CA60701A9B6A19A8B523EA0DD9A300516
:108F1000DF991CB9DA7E26CEB9E4A1B8BF90F20081
:108F20001ACFBC037532CEE167052C6527D0E1036B
:108F300074023CE7DBA4A7D8DEA708C56801A53EFC
:108F40005347982BB0A6694784D694FB418EA70758
:108F50003A0E5A6AFDCD14F6C1E2141B2815E71D1E
:108F6000A10E5CCDD9D4E8AC6C5C431409A159CFF7
:108F700061177FD45F818AAF1B45C4F5EFA51CCD77
:108F8000E1A1AB59B742A01F7B692328636BFBA803
:108F9000F5A05A5E397EAA8B97364DD2B6BDE0DB7E
:108FA000AA49921FFAB0D238DAF116F32A84550B87
:108FB00007F341F91B8D3C4CDD84DE3F7A7ED77E82
:108FC000F800AA8219CAFB276A311C07E2CC1A9D55
:108FD00051F1BE4754FB8CEFF5F1C9A7AF41229385
:108FE000954E2F99E02E2D13F03526459014A5327D
:108FF0006C10A2346E2ADE85D859DD9D2B4CD8EF3B
:1090000021DE68652E77B21C564C50BF6788B78347
:10901000462ABD1D42BB21A16F918E4411E648B185
:1090200047CBDB360FB9F0C3A6F9B0A4FC2FFCE0A8
:1090300018472B35AF8BFC8F8C4102CF55F25DBEAC
:109040001659D844F9158E4D570947A1D28D2DD503
:10905000ACF9C89C9183B6FAB95F5A3EEE4D7801DF
:10906000027E7880C0DB092CFE4C1B677350B6BAB9
:109070005C0F71E04D36FA026B1293D0E1A73939DB
:10908000DAB4A050C1CA160BCEFD308B3714DB0BFF
:10909000618D6377669EF58F7D9B75B2A080FB8F97
:1090A000374358251DFC77D033BF75430E1A1E1960
:1090B000529FD2F0E5EB04D57B684DAD654C33860D
:1090C000D06EFC40DA19B655DA948F0FC06336FAC9
:1090D0007E087B2E0D55912EAA0775F4B5F3D24A62
:1090E00008E9A41F1C2F29D2E50EC5F0662596AC11
:1090F0002E13F2748104E986B65269068584E5FB75
:10910000C73B54021EF957273121F8D867B6189E7D
:10911000C43AA1F848C23DE6F0AC946BC90FE31F16
:10912000A30F8626B8DEC85A64724E281E4821B4A2
:109130004CC77809EBA5F80281B17C94D6B15CC12B
:109140003C4934FF98F3F84BDC0146B66398AFD046
:109150002AB629E8D0633590026E5BADB0E2DE75C9
:1091600036FB6C7F94B601A7DF06E9EC4D2AC9D126
:1091700066D4DEDE6A98351D1C771241ECED67ADD2
:10918000C53B6BC025DD25D8B53D154848A5FD6814
:1091900098C09FFBD3A0E07CFF4B479143F921F39C
:1091A000E14D4ABBDBBE996653006EC8C5D4DADE1A
:1091B000C2F8DA959E09588FB3FC322410E2DD9B89
:1091C0002560602F62E4737B0083E7298983A0C355
:1091D000C9D8EAE0959F81CB78A23F4FE1C18407CF
:1091E000ADFE03C3FBAB3A4DB13E8422F072603258
:1091F0005A3D536772D921AF745616ADDB38FFAABA
:109200005D1CFB9DF21D84A36C5E24F56323F43E7C
:10921000BBFA61E50038ED8A2998F426EF3233E095
:10922000148698972E9BE87EFB017E431A5B4021B3
:10923000EC5878A142729A2EBF412D9827617B137A
:109240005BC85BEADCF450BDBEE3D585011EB7D830
:10925000A1FB5F201C27C18BC4B72E78636862FE18
:109260008FD2F353E2532769D56BEC4E6F7CD52F29
:10927000277F844D4727CDB3B37F7E6E24AEE7A50D
:1092800064D30F531704DB17C7FDE5673297EAACC9
:10929000B1A84B02C40941CEBA4A4B58009DF8917F
:1092A00011AC527820068A29F62CA18864FCA837D4
:1092B000481EBCEAEAA8F640A799393564DB9C242D
:1092C0000248E94C6F40CB1EEB979F381983FBBADD
:1092D000A80AAC1E45A14EDB1021651F78A716B663
:1092E000D521443A51D46BB88552A17A61FFD43963
:1092F000C883AEFB9AE6CFC7E45A68D43C64437691
:109300005509BCB350168FB6325C65093F4D925B70
:10931000534F9439FE4AA4AAD1447C022DC0B7BC55
:10932000D9292365C54821D39F5810F49AC3ECF579
:109330007E6CA1800EAF7F24541CAB2F64EFA13E46
:109340000D08CE5628C20AF97539298B4E52AE89BE
:109350006BE74A28D1CD52FFDC8957904AB89F1E4F
:10936000CC38F5D1BEEABDED431526D91E1367975B
:10937000DC3929B7B7FCBAE7EACD1985EF726ADDA7
:1093800083768AB2CDC7FE0719124ECCC83A952D06
:10939000EA5AFBAD98BE96BD22ED5E72563AE224C3
:1093A0005E2F8905A52160484C22BB89E0B49F82CD
:1093B00002A956B1DD081D44466D6E5F48C6ACA9D2
:1093C0008ADD3FC126D57C6AA327F80D4A335D4765
:1093D0006D2058303AC5C0CDE0B8A1E1B74BA49C90
:1093E000AF07E6E757C7047090718E935D7792855B
:1093F00027293852E9A9FD8C9EE7AA8AC77FEFF199
:109400006653F634BE0B26386B2CFB39153BCB95D7
:1094100065B283F9C25B03670CE7FAE559FC2E2FAE
:10942000543EA6E4E26EEA33A5B5DCB3B53207AC30
:109430000A1D7618D131D71BA4AB557C4F0F3611BE
:1094400069D1DE066AB7FF392F04E1D7E2F8026A74
:10945000925B62BBC63C8E28FB54DF74C649B17B6D
:10946000B1F7E62F1801712CC83F2CFF7390ABDBCE
:10947000A85F68D7FEECF66018FF11E190D999B9A2
:10948000CAB62040750E4AFEC72B8D5F0186E4F5F3
:109490005A266B012619E26797ECBA98EF0905C9BD
:1094A0001FFE179D9C827C117CB844C8080AB647F1
:1094B0003B77B691290A4ACDEBF8E3A91A7C4AB763
:1094C0009663C84920F65997268C376166EEFDED04
:1094D0004A409870F8B1D7DF08AA3D683FECFC8A93
:1094E000314967E3AF796A7FD86987F6382D4E39FD
:1094F000E6DB7D96A2F897414D734A240AB47B506F
:10950000074A420778AE4029FEFDC091C33D777AF5
:10951000C3690D7C7C2A39F0138A2B78DD7E541ABE
:109520000766A5A2CD6F030F883653883A16F60258
:10953000DC8B2E8B7D8F83A88756B5149FA99FF156
:10954000AFA2C0FFB0940841D91393476F6FA491A5
:10955000F2974C9CCCD15D274FD06CB42C4FBDE61C
:1095600025DC69C41079F09A59B2843A3894606461
:109570005ACC4B818AE5E88042DCC56A6612280530
:109580005AA52AC72B810B8D1637AFBE6AC43ABACB
:10959000A889E5DEDD2082F99E860A3600DFE988AB
:1095A00081D86AEA11BB50844AB61D2045C8EF81B4
:1095B000026D66C7BB27E2F6C16F7D4E181AB21E58
:1095C00087E2E9243B5ECD847ACB67CA6D62C252E2
:1095D0001AB065734B363CBE5D417F984087BB7DBA
:1095E0001B4BD1B53AEB3DA07D1420405239DAFC3B
:1095F0001548FC3D521250938F91A886A9BC182F94
:1096000010A1601C1C4FD93347BC066C240D486F59
:10961000D30B87B55D9BC2C066178310177679534D
:10962000D0C320DF314C1F29AE3814E07DBC146458
:109630001AF5E235C1AAFF36AD037019F3F2BA1775
:109640005E377A73EF3F9732D0321DEBC78C70EDE7
:109650004E36193D0F38A40FA46FA296D24983E568
:10966000B8B241A29BD00B5D2299242523D4A43407
:10967000E43328AB3AA4EDD15596082CEB4D81404C
:1096800047FB9066A53993E47B309A056567DA5904
:109690003B997256497B75F4EB1681F486DC7ED0DB
:1096A0002ACC4A24F5F380023E8CBEF1B92B325EFF
:1096B000DD02B0EB4EB65503EC5C841121F2262A94
:1096C00004DDD86A7D00E206FD73FAA11D5AD8EDCB
:1096D0005130562DE34953C1865957021305F6F40C
:1096E00041BE3A30E90C85398A1D983805048EF35D
:1096F000642C196CCA66387288E78E75EABB7C9B4D
:10970000166D86513C7E53BB5A257F31E353208032
:109710006FAA66D5D2882D71717B9A486C7644DB2E
:10972000940A8489F3F777E173DA937E2E34DB1F92
:1097300071183E417E602420A8E54B2678CD53AEBB
:109740002DF31E019A594EE04AFE93A259C67EC8D7
:10975000C76CB0B83454907406ECD82A18AAA61571
:10976000CB568274B4052F418F6AB6F3974A79E1DC
:109770000585319EEACD50D006516F8C45AA05680B
:1097800060AE77CEED655C6C264217920AA4BC37BA
:1097900072E96D4C0F34B78209273C72AA85E1A3A8
:1097A000B7A6219194BD9930C5CC7D443D6E33D090
:1097B00092059B2233502DED55066AE4E7032A10EB
:1097C0009ECCAFF116051E21B47C8773EA89AECC1E
:1097D00088368832F31FED2DD5B76933109C9B7006
:1097E000102EF446447D6438628B18D59C6F3FE29E
:1097F00069B5B9235CDF4B3102F6BB9A34D64A49CE
:10980000DEE1564E46507951F8A7E1C60E822F7B15
:10981000B7367B744BA3019C2E172C0DF19D1E4374
:109820008665FBBD8F251F11A3383D42A4195E1428
:109830001802BA3F14B1DF35F68594D03071375A2B
:10984000BECED433D15BEB9ED6C8260B827073C9D3
:109850005786C2590C6B1606F54BB567F452F69E47
:109860009FBC46B1308CC1ACD9E4A32332D29A322A
:10987000FF311AB247F98F6864FB3FF105BD0C93C5
:109880009E6C79AB72FEC8236BB0A72D517DB78F4C
:109890005C1004819CE895A737FB4E2D4FB6B91C90
:1098A000DD21663570FCF2371D78AF9DDFE73CBFE8
:1098B000A0239DCDF796457298BF9937B710819C2C
:1098C000E0F2C36EABBE03ABB7D12218FADEA277CB
:1098D0005B3AFB55A0F6831FFC89AA89939BDD6246
:1098E0009F21E0FCB5F430614DF606485F4ABE7535
:1098F00002E492967D36C8807175A23F7F7B37CC9B
:109900006E021737B85A59C37E0004E8D6FB0D7FA4
:109910009C3CDFCB6B1B7818FE2122B00067141E25
:10992000E4DB6D0B99173683EA42AE9B555C1A5700
:109930004550871D20578EB3FB384E80255E2DACD9
:10994000969CF078BF7E57423126EEBF202AA3872F
:1099500002E49A1C3231B6BCC6922A13151AB27CA4
:1099600082A7D25BBAFC2E6D98A4EB9C45B14A70DD
:10997000FBBFF334B8F2BA0AFDC334B41C459F40B0
:109980007B95F6B111A81A0EBF3F012D857B21A949
:10999000C7F25E3B896C1A447E11602816CDBA73FB
:1099A0009C40B1596BAC2C96C3EC20FF99D65AAEB3
:1099B00085EE4BF7C51EF5B6C3144A0FA76D44A636
:1099C00044FF574B0D132FE97E72BD8F10111659AE
:1099D000BE6C9CE9099C2F09767E0415478E48923F
:1099E000C861614759A7D671B849ED6B754AF82A25
:1099F0005A4F69375CEC5C64F13F1DAB9802DE198D
:109A00007C97DB53E131D9D79CD3A799CF33571239
:109A10001D951B911F0653FDDCB01D38CA121ECFC9
:109A2000C2833975416D1C6A25B3AA35B3346236D9
:109A3000371557F29EC1E089D15BBA46BD3B923FD4
:109A4000DB2CD0A2DBF83AC2AE0E10AC8D87CA2F49
:109A50005EE6402CC27AB699CE14F0884F2D9668F7
:109A6000F976D5073E3B5AC932C840CEEE65A415FB
:109A7000316AE92211F1F117BF8021DA9D2CA2E8A9
:109A8000E26F7E3A8ED8F2C3F54B34788A75F28A4B
:109A9000BB8DA9E0F9C718A80AF8406394AF481035
:109AA000F1808D9CB121785420C5EB35CB3BC89A11
:109AB0001C5F0E222B12AC17B249E0326C2A034411
:109AC000A35575326440F6EC56AD7190C26556A64A
:109AD00013AE2E30D5476BFFEA1CA842EE20609CE7
:109AE000FFEEE2D7B04A1C7C8E691F64C9E5C566EB
:109AF000FDB9DF53F931F2FFB707C15980993B1C1B
:109B00004C01307D101FDC72DDB8D2D6D41B4F5C07
:109B1000E17B84959B910BF6D11F9FBD9485FF033C
:109B2000D4CA9B9014867F314D9197B21756080284
:109B3000F84197E841A933F99A2B2BED1E3AB3B9B6
:109B4000FB819F8137C519EC9946F5D96D8EE85E8A
:109B50009DA9E4125751E887A12B07CE518C160915
:109B600032E7C291FEA66E44A79EA3C4470ABB502B
:109B70001216CE7B446E2FDBD87A4D8CEDFF302E43
:109B80007A8E701EDDF300D13460E2818AE26B3A96
:109B90006862FCA52832E2F7285EADC21DAAED1F5F
:109BA0008719C38A6D7750ABCAC198FBEDFCE703F8
:109BB0005848904ECD0CA180397B3FB2EA53AE8C11
:109BC0001D33A72F70135DA52232DFFCF4F56CEA7C
:109BD000794C76A1EC25030F7C6E7134DFA578BF3C
:109BE0007F50958D6C395CC448158DB958007095BF
:109BF000F7CE2C385D37F2E9670CB8D31D3B2D82C8
:109C00004FEE42436FDFE389C5281D3B3896233B67
:109C1000CC3362A2AF86D35537CEC84093FB1F2901
:109C20000CF8F4E7F0EF38766FE53B2CB7BA4774E1
:109C30006D1CBC08CAE24622A85FD85AEA0A9F54A3
:109C400054DBA8EF882F2D55FE3723CC5AE5F07151
:109C5000EAFC6C939095F6D8AB36CEAE6DEB07B2BE
:109C60001B559E0808AE0E71F2B57419B0EE87D37D
:109C7000625B7743624EBDE65D316C07ACDB22531D
:109C8000B3C2F0FE68C692D61EDEAC3A7926B2D2D6
:109C900061A939A73F63F4A6233EE4A60A8C628437
:109CA000BA05D331AE1F8AD4A2B361CA664C24DE92
:109CB000BEB50A0503F85E3F67232CC83DE4D06AB1
:109CC000C314E408EB56CF3907BBAA4DA2B288FBF8
:109CD0003FAE7D1D3931E5EAA416A5F970609CBA46
:109CE000E7646C956DD4C1CB00C81AF5C2EC65274A
:109CF000AF7145BA1D62C9AEA212D0D4B3BC840AFA
:109D0000A37DB78F664853586DF58CFAD2CFC6FD48
:109D10005A5011062048B6145604AE51F4F6B881D4
:109D20004D15706716AD0BC3EE9753CB0ADF832535
:109D3000B18EAA42A94DD7BEF24FC35C3652A79549
:109D4000CDF87A07110A352A03E4B1559F44F80F7C
:109D50004F75E13A840B11E0D8CF058623A0745FDC
:109D600056AEC5D13766A484FADBBAE8C6E1B00ABC
:109D700065027FE6222FC6FA6ABE30E1D748FFC2ED
:109D8000DF9AB35C065CD2D4A681E4BB11D8BE1FB7
:109D900006B467F9B51BA7953CC142C5660530708E
:109DA00086D2E7D2C238F0775A617116E03E17309A
:109DB000A22923F2318415A4412EE78123ABA4A26A
:109DC000F6FDE466F5686D7CE078606B300068DA7B
:109DD0007DD7E00F1DDA7A6D4A378811A7DA19624C
:109DE000C8084418DB14D3DAC954F684D6D9AC8138
:109DF000CED83891FC98772D28AC41D10C2A36FB6F
:109E0000841591486E387EE764E14E51687CF269B2
:109E1000865BFF1F7141D7757346FA5008326ACCD2
:109E2000E41C03CA4D1938A3476DF3184103360AE1
:109E3000F6BAC1E06E29AF85F03AEBCD222DB3D74B
:109E4000C9E6C2E4DD438AB0FBF3A64BAAA594960B
:109E5000C416426A5828F72E4CEA832D495A53AC4F
:109E60005042D286F4160E348F06F0ACE0C4247B48
:109E70004A883E03FB240C83FA62533A1F18BF1B27
:109E800009E5C14400CBB3BA0E63CB7925DAF12ED4
:109E9000D9E701B5DF3623892DD63ABB3FC2691D0C
:109EA000B2434560EB2EBF24FEF546856830547DF5
:109EB000A9C74909F1741CA628BA6C897CFFDCDDAE
:109EC00082CFBBF32F3C0B2A225FE1A6C791CD14B2
:109ED0009B530B5C79CDB1996896E2DC0950F5A4EF
:109EE000DCAB2287B1FFA39C04C7748319D2A30AF9
:109EF0004C58ECD197587B84590A0554C8B1C5C257
:109F0000DA52AFCE3C1D5FCE2AADF3B3016B2E9378
:109F10007B3FE77A9BB8EFDBD41A981C1A477E295F
:109F2000BC25C3B9FEE196EDC4A8639661B4DDF526
:109F300052B868887E5A91BB8BBF7DC58F77849C51
:109F4000EB1A36FA7345497955AB904D7A8F8505F2
:109F50001E2036763095D5EC85BFE9C964F3A8BDDF
:109F60002F211BA15E0D63D4D1DF3F474CE512CBFF
:109F7000F72FCDF7B9D7255BE41990C0CD82EB4020
:109F8000F914ADAD5C9A6D632BD1724201E5152ACF
:109F90007C66D9851C2458D8431D7A76F7D129B818
:109FA0001FB1F4324AFF0763ACB489A08730A631F1
:109FB0002CACD29CEAB9BAB4CA73A23378F46FCD90
:109FC000F5195A973D762DF7BE79F01B80A7EBA0C7
:109FD000DEFC94BC5295DCDFFC9275D9FBE60FE108
:109FE000189070F2845B729E63761898B656E1C33F
:109FF00044DA5C9541B0367BDA57F016459ABB1FC0
:10A00000877DEF940659C637FD2694038211F4E14B
:10A010001E0D272249AA1367C8DEFC88A99F5DA6EA
:10A020004B3E1249C794DCCFD6492A73503D4FB6F8
:10A03000494702CB528FFB20F376CD0268AF905098
:10A04000D8B6B368E3B7318FD82E121E1998AA0F6D
:10A05000FCB10B6D0A78F414D2C445C4169ADE6FB5
:10A060009E6300326839BCCEE62605880D6B79F216
:10A0700044038D201175C5E84AEADC92DAAE0ABDC8
:10A080003A5AA11B832C56FEAA63D33C69EEBEDB71
:10A09000217453C66A98AE262F78618DAE3B861B1D
:10A0A000D268F2BD31A6642F6773B60595E73A769C
:10A0B0006197B879E1C728CF617A74382BDF5C5893
:10A0C0005AB94AAB13F9386A958BA213E6B178A94D
:10A0D000E6098190227CB2AE47CFC94DC1A332932D
:10A0E000983B2FA71C6E1066C989804B4D2CC49ECF
:10A0F000C1B9C548853CFE4820D05227FD4A66AA12
:10A100000304050A08060BFF0209070D010C00FFF6
:10A110002025692025692025692D25690020202515
:10A12000633A256900202020205F5F7C002C0061BD
:10A130000044697370206F66660D0A0055534552DE
:10A14000004600424547494E0052414400442E4DCE
:10A1500059005052474D005553455220202000666B
:10A1600020200067202000424547494E2020202023
:10A17000200052414420202000442E4D5920202010
:10A18000004320202000081C242C4448586C7403F1
:10A19000050000FFFFFFFF4D000000FFFFFFFF0F66
:10A1A000000000F401000004010301020101041198
:10A1B000040F04170416011801000057A100005FE6
:10A1C000A1000063A1000067A10000EE570000722B
:10A1D000A1000079A1000081A1000052A1000005AA
:10A1E00002050804080B0804040501050409080910
:10A1F000040608070206020402060106040701031A
:10A200000803040C080D020C0203020C010C040DDF
:10A21000010D080D040802080807080202070408D7
:10A22000010804090209010A080B020A0201080ACE
:10A23000010A040B010208020410081102100211A5
:10A240000810011004110112021201130213081266
:10A25000080F081204130113041402140115021547
:10A26000081408170814041501150417021701191A
:10A27000081A0219021602190119041A0116081601
:10A28000041B021B081A0818021A041B011B0418DD
:10A290000818040B0420202020202020202020004B
:10A2A000000000030000003CA1000041A10000EEFE
:10A2B00057000043A10000EE57000049A100004DE7
:0BA2C000A100009F64000052A10000FC
:00000001FF
